:10000000F01F0010853800008138000081380000A2
:1000100081380000813800008138000000000000B5
:100020000000000000000000000000008138000017
:1000300081380000000000008138000041160000F7
:10004000111400001114000011140000111400001C
:10005000111400001114000011140000111400000C
:1000600011140000111400001114000011140000FC
:10007000111400007D3800007D3800007D3800003C
:10008000F9160000111700002917000041170000A1
:100090007D380000091800007D3800007D38000020
:1000A0007D3800007D3800007D3800007D3800007C
:1000B0007D3800007D3800007D3800007D3800006C
:1000C00008B500230B60036000F024FE08BD08B5EE
:1000D0000A20002101F0B0FA08BD000038B5094B34
:1000E0000D1C041C1968012001F056FB012001F0D1
:1000F00033FB291C201C02F025FF012001F03CFBF2
:1001000038BDC046B004001070B5054E051C0E2465
:10011000013C295D301C01F099FD002CF8D170BD27
:10012000B43A000038B5164801F090FD154C201C7B
:10013000FFF7EAFF144D4221281C01F087FD201C27
:100140000E30FFF7E1FF4321281C01F07FFD201C4A
:100150001C30FFF7D9FF0D4801F078FD201C2A3034
:10016000FFF7D2FF281C4E2101F070FD201C383013
:10017000FFF7CAFF616D064801F068FD38BDC04653
:10018000B73A0000B8040010BD3A0000C43A0000BD
:10019000CA3A000008B5074B0120196801F0FCFAC3
:1001A000012001F0D9FA02F065FE012001F0E4FA25
:1001B00008BDC046B004001010B5041C0D2107484E
:1001C0000C2200F0B3FC00F013FC201C00210322E1
:1001D00000F022FD00F016FC10BDC046553C0000AA
:1001E00013B59620000201F04DFB1248FFF7E4FF23
:1001F000FFF7D0FF1048114901F028FD002401F05D
:10020000E7FB002802D001F01DF800240A2001F0CD
:1002100043FA684601A9FFF753FF009B002B03D167
:10022000074B01349C42EADDFFF7B4FF054801F0BB
:100230000DFD13BDD63A0000E53A0000F03A00008B
:100240006F170000FD3A000000B5074B89B01A781F
:10025000064B68461B78064901F003FD6846FFF728
:10026000ABFF09B000BDC046B8010010000000108F
:10027000083B000013B5FFF7E7FFFFF78BFF0024F3
:10028000684601A9FFF71CFF009B002B2CD0182B00
:1002900021D004DC142B0DD0152B20D104E0342BFD
:1002A00012D0352B1BD107E0134B00241A783E2ABD
:1002B00016D806E0104B08E0104B00241A78062AE6
:1002C0000ED801321A700BE00C4B1C78002C07D0B2
:1002D000013C1C7003E0FFF75DFF282400E00024D0
:1002E00000F072FBFFF7B0FFC820013401F0D4F931
:1002F0001D2CC5DD13BDC046B80100100000001064
:1003000073B5124B041C1249186803F03DFB1149E8
:100310000090114A114B201C01F0A3FC00F0DCFD01
:10032000002812D000F0F4FDFA218900051C03F02A
:100330002BFB061C201C01F0E1FC094B2018734329
:100340000849EB18321C01F08CFC73BDB40400109A
:1003500040420F00163B0000F03A0000233B000033
:1003600018FCFFFF263B000070B50D1C161C041C7A
:1003700000F03EFB0B480D210C2200F0D7FB281C9F
:10038000A1B2002200F048FC07480321062200F039
:10039000CDFB301C0121092200F03EFC00F032FBB5
:1003A00070BDC046553C0000923B000038B50D1CA6
:1003B000041C00F0E8FA2A1C0120211CFFF7D4FFDE
:1003C000034B00225A60034A943212689A6038BD87
:1003D000540C0010B804001010B588B0041C684616
:1003E000FFF78EFF69466A46201CFFF7BDFF08B085
:1003F00010BD000073B518200021FFF76FFE424EBC
:100400000024424D983600E0404D012001F0B4F93F
:10041000002C01D0002000E00620012101F00CF9A1
:10042000684601A9FFF74CFE009B002B21D1002C50
:10043000F0D13368002B0DD0354B00941A6811327F
:100440001A6004E002F0C0FC009B01330093009BA3
:10045000102BF7DD2F4BED18DED518200021FFF70C
:100460003DFE294B94331C6863425C4100F074FAF2
:10047000CEE7002C03D0182BC7D100F0CBFA009B9D
:10048000182B2BD1019B00220192822B22D004DC5D
:10049000322B0ED0732B20D119E0832B0FD0C22B1F
:1004A0001BD11D4B196801311960022916D11A6040
:1004B00014E01A4B01201B68C01A00F03BFD01201C
:1004C000FFF78AFFFFF766FEFFF701FE06E0FFF782
:1004D00087FE03E0FFF7CEFE00E00193104B012002
:1004E000196801F059F9012001F036F900980199D5
:1004F00002F028FD044B002494331B68002B83D1A9
:1005000000F02AFA01247FE7B804001020BF02009F
:10051000E40200100CFEFFFF900100100800001024
:10052000B004001013B501F019FC00F0BFFB00F09F
:1005300071FA1C48002100F01FFF00211A4800F04A
:100540001BFF00F059FC00200421012200F0A2FE54
:100550000020021C042100F0EBFE002005210122F6
:1005600000F098FE00200521021C00F0E1FE00F0E2
:1005700075FE3C24201CFFF72FFF013C1E2001F0DC
:100580008BF8022CF6D102F041FB1E2300930F23BF
:10059000019306480649074A074B02F0F1FBFFF7B3
:1005A00029FFC046984004409C4004403938000070
:1005B000C1000000AD030000E402001000B500E03F
:1005C00001300378202BFBD000BD00B5031C303B6D
:1005D000DAB2092A01D8181C08E020231843031CAA
:1005E000613B5738052B01D90120404200BD70B551
:1005F0000E1CFFF7E3FF0025041C06E0FFF7E5FFF4
:10060000002805DB2D010543013420780028F5D1B1
:100610003560201C70BD000008B500F079FC011C9D
:10062000014801F013FB08BD313B000000B5C300D9
:10063000181A064BC0180723013BC25C002A03D1DD
:10064000002BF9D1012000E0002000BD540500106E
:100650007FB5194801F0FAFA00250326354219D171
:10066000281CFFF7E3FF002810D0681CFFF7DEFF0F
:1006700000280BD0A81CFFF7D9FF002806D0E81CE3
:10068000FFF7D4FF002801D004350FE00B48291CE8
:1006900001F0DCFA291C684601F0CAFB6846FFF746
:1006A00033FD074801F0D2FA6C1C251CFF2DD5DD67
:1006B000FFF738FD7FBDC046F03A00003D3B00002B
:1006C000097E000070B50E1CFFF778FF0D25041C95
:1006D0002078FFF77AFF002807DB01347055013DD1
:1006E000F6D2201CFFF76AFF00E0002070BD00007A
:1006F00030B5464C87B023680868002B06D14448C3
:1007000001F0A4FA02F082FA012357E0012B12D182
:10071000037B202B07D0002B05D03E490C2201F093
:1007200000FB002803D1394B1A6801326AE03A48CD
:1007300001F08CFA5EE00378412B1BD1374C02307C
:10074000211CFFF7BFFF002854D00378422B51D162
:10075000211C02300E31FFF7B5FF00284AD0037884
:10076000432B47D1211C02301C31FFF7ABFF00287F
:1007700049D13FE04D2B23D1294D0230291CFFF7F1
:10078000A1FF002836D003784E2B33D1291C02302C
:100790000E31FFF797FF00282CD00378472B29D183
:1007A000023005A9FFF723FF059B002B22DB2A3D22
:1007B0006B651C481C4901F049FA0023236022E0C4
:1007C00005A9FFF714FF0378041C202B01D0002B90
:1007D00010D10025201C01A9FFF774FF0599041C06
:1007E000691801A801F038FB002C03D00135042D55
:1007F000F0D108E002F00AFA0A480C4901F026FAA2
:10080000024B00221A6007B030BDC046BC02001087
:10081000463B0000F03A00005C3B0000B8040010CA
:10082000E2040010683B0000723B0000753B0000D2
:1008300037B54C6824E0201CFFF7C0FE01A9FFF784
:10084000D6FE019B041C002B1DD0D8B2FF2B09DD66
:1008500000F0FCF9051C01980012C0B200F0F6F996
:10086000019003E000F0F2F90025019001980028C2
:1008700002D0291CFFF732FC23785A1E9341E4185A
:100880002378002BD7D137BD08B5064A012113784C
:100890004B40137001D0044900E00449044801F0C2
:1008A000D5F908BD9D0300107C3B00007F3B000094
:1008B000833B000070B5051C01200821021C00F0DC
:1008C00037FD0724012601200821002200F030FD19
:1008D0002A1C224132400020022100F029FD012083
:1008E0000821021C00F024FD013CECD270BD10B5C3
:1008F0000021041C0A1C022000F01AFD201CFFF736
:10090000D9FF10BDF7B5012300930023019372B600
:100910006C46061C02AF01CC50235B421843C0B2A8
:10092000FFF7E5FF0020FFF7E2FF1020FFF7DFFFF2
:10093000E020FFF7DCFF002502200021012200F06B
:10094000F7FC705D0135FFF7B5FF842DF4D18436D7
:10095000BC42E0D162B6F7BD08B5AC20FFF7C7FFD7
:10096000AE20FFF7C4FFA520FFF7C1FF08BD38B5D3
:100970000D1C041C012200F08DFC291C201C0122EE
:1009800000F0D6FC38BD08B5AF20FFF7B0FFA420BB
:10099000FFF7ADFF08BD08B5AE20FFF7A8FF08BD03
:1009A00010B5041CF820FFF7A2FF201CFFF79FFFE3
:1009B00010BD10B5041C8120FFF799FF3F20204097
:1009C000FFF795FF10BD000008B5074B20201B78EE
:1009D0001843FFF78CFF0A2000F05EFE034B1878E7
:1009E000FFF7E7FF08BDC04600000010B801001087
:1009F00008B5842202480021520001F05FF908BDC9
:100A0000A503001008B50248FFF77CFF08BDC046EB
:100A1000A503001008B501200821FFF7A8FF00205A
:100A20000221FFF7A4FF02200021FFF7A0FF022010
:100A30000621FFF79CFF0320011CFFF798FF03200E
:100A4000011C002200F074FC02200621002200F0AC
:100A50006FFC06210122022000F06AFCFFF7C8FFAC
:100A6000FFF7D0FFA220FFF742FFA020FFF73FFFD4
:100A7000C020FFF73CFF0020FFF792FF0A2000F0A4
:100A80000BFE4020FFF733FF2C20FFF730FF322012
:100A900000F002FE2E20FFF72AFF322000F0FCFDBE
:100AA0002F20FFF724FF0A2000F0F6FDFFF78CFF50
:100AB000AF20FFF71CFFA420FFF719FF08BD0000BF
:100AC00000B50F290ED883280CD8CB0884225343B5
:100AD0000722C0181140044B80220A41111C1A5CE5
:100AE0001143195400BDC046A5030010F0B55B18B2
:100AF000DBB216E08425CC086C4307270F40802525
:100B000004193D41EFB2A6189C4605E0064BE518D6
:100B10002B7801343B432B70B442F7DB0131634641
:100B2000C9B29942E6D3F0BDA503001000B5074B4A
:100B30001860074B1970074BD1081A70064B1970D3
:100B4000500701D00131197000BDC046A00300104C
:100B5000AD040010AE040010A4030010F0B589B07D
:100B6000059106925A2800D92020284B284A1B6854
:100B700093420BD1440003212418623C019103915C
:100B80000EE0195D01320231641802E00024221CDB
:100B900020388242F5D31A5D1B195B7801920393CA
:100BA00000252CE06B430199FA188A4215D2174AA6
:100BB00000261268D2191219D3189B7804930123C6
:100BC000049AB340134205D0029B07989919C9B201
:100BD000FFF776FF0136082EF1D1029B013708336B
:100BE000DBB2029306E0059A06995319DBB2029133
:100BF0000027079307490B789F42D3D30135039A07
:100C00009542F0D109B0A8B2F0BDC046A0030010D3
:100C1000923B0000A4030010F7B5061C0C1C0192C7
:100C200001F06CF800250090832708E06B46705DAA
:100C3000E1B21A79FFF792FF013024180135A7427B
:100C400002D3009B9D42F1D3F7BD000000B50F23F6
:100C5000020918408000031F00D52833002B0EDB4B
:100C6000511E0320884280414042002807D1242B96
:100C700006DC04218A1A0349CB18985C00E00020A6
:100C800000BDC0465840000070B5064E051C00244B
:100C9000A05D054B291CC018013400F06DFB0A2C27
:100CA000F6D170BD9440000000400440F8B510201B
:100CB000FFF7EAFF094C271C143725786678281CB3
:100CC000311C002200F0E6FA0234281C311C0122FB
:100CD00000F02EFBBC42F0D1F8BDC04680400000C1
:100CE000F8B50B4C271C143725786678281C311C66
:100CF000012200F0CFFA0234281C311C002200F03F
:100D000017FBBC42F0D10020FFF7BEFFF8BDC04684
:100D100080400000F0B589B0002404900591FFF7F1
:100D2000C5FF0220072101220694079400F0B2FAC1
:100D300002200721221C00F0FBFA201C0B2100F0EE
:100D4000CDFAA04202D11823069301240021264D9A
:100D500003916A782F78111C0192381C012200F04F
:100D600099FA381C0199002200F0E2FA03231F4E81
:100D7000029314E03078717800F0B0FA002807D1BF
:100D800003991B4AA3008A5C183369465A50013400
:100D9000029A039B013A013302920393023EE30F4E
:100DA00000210122A2424B41DBB28B4202D0029BC6
:100DB0008B42DFDA381C0199002200F06BFA0199AE
:100DC000381C012200F0B4FA0A4902358D42C0D124
:100DD000201E06D0069B049A05991360079B0120EC
:100DE0000B6009B0F0BDC0468040000056400000D6
:100DF000584000009440000008B50120021C0B215F
:100E000000F048FA01200B21002200F091FA0320A3
:100E10000221012200F03EFA03200221002200F00C
:100E200087FA08BD37B5234B10211A68051C8A4381
:100E30001A60214B8022196892010A431A6001202E
:100E40000B21002200F026FA01200B21002200F0E5
:100E50006FFA1A4B9F211A68194C8A431A601A6854
:100E600018491A60184B186802F08EFD80230002A2
:100E700018432A1C20600221032000F059FA142094
:100E800000F00AFC2368FF229343236023680F4A83
:100E9000134323600E4B1A680192019A002AFADA72
:100EA00022680C4B13402360FFF7A6FF0198000453
:100EB000800D3EBD3882044080800440984004404C
:100EC00000C0014000093D00B40400108000000192
:100ED0002CC00140FFFFFFF810B50C4C2068002823
:100EE00013DA00202060FFF79DFF0A280ADC0120AA
:100EF000FFF798FF0138C023FF385B00984201D804
:100F000001232360FFF778FF206810BD0400001064
:100F100008B5FFF7E1FF011E08D00120FFF782FFAF
:100F2000011E03D0024802F02FFD011C081C08BD61
:100F300050BB120010B500280DD0254B80211A6837
:100F40008A431A60234A012311681942FCD0224BBC
:100F500003221A6001E0204B1860204B012200217F
:100F60001A6019601A6019681142FCD01C4B0122EA
:100F70001A601C4A802114684902214311601A1C1E
:100F8000002804D1124B8024196821431960164BA4
:100F9000196888421AD01860002801D0134800E070
:100FA0001348116802F0A2FC124C2121206002F0CB
:100FB000EBFC114B18609620000200F063FCFA2154
:100FC0002068890002F0E0FC00F04CFB10BDC04638
:100FD000388204400C8004407080044074800440D7
:100FE000788004408080044008000010006CDC021F
:100FF000001BB700B4040010B004001008B500F0E6
:101000003BF9134B00211A68120B12031A60114BA3
:101010001A68120B12031A600F4B1A68120B120394
:101020001A600E4B1A68120B12031A600C4B012245
:1010300019600C4B1A6019601A6019681142FCD0D3
:10104000094B23221A600120FFF774FF08BDC04638
:10105000008000500080015000800250008003504A
:1010600040800440448004400880044070B50F492B
:101070000F4800F0EBFD0F4800F0E8FD0E4E0F4D5D
:1010800000242B196159DA68301C0A4B143400F023
:10109000DDFD782CF5D10A4800F0D8FD00F018FBF2
:1010A000011C084800F0D2FD70BDC046F03A0000B7
:1010B0009E400000EF400000AF4000000C00001018
:1010C000BA400000DC400000F0B53C4B8BB01D681E
:1010D000002D3AD03A4B02901B6801209B685DE0DE
:1010E00001342378202BFBD0002B3AD0B3000833F7
:1010F0006A469C500136FF2D01D135E0013423783A
:10110000202B01D0002BF9D1202B02D100232370FA
:101110000134012E1BD12A4F2A4B07223B6001923A
:101120003D1C09E02B680298196800F009FE0028B0
:1011300008D02B6814332B60019B013B0193002BDB
:10114000F0D132E03B681D7901E0041C2E1C2378AD
:10115000002B06D000230722B2425B41DBB2002BFA
:10116000BFD1002E1CD000E00025154C022E05D169
:101170000398154900F0E4FD002801D0AE420AD8DA
:1011800023681248D96800F061FD23681048196986
:1011900000F05CFD04E02368F0B29B6802A9984768
:1011A000064B1B68002B07D103E00198011CFFF7D9
:1011B0005DFF084800F04AFD0BB0F0BDBC02001016
:1011C000C40200100C000010E9400000EB400000D9
:1011D0006D3B0000F240000038B5041C154D0A2894
:1011E00008D002D808281CD110E00D2802D07F2892
:1011F00017D10BE02B6800221A700F4800F026FD73
:101200000E4C201CFFF760FF2C6012E02A680B4B8D
:101210009A420ED90A48211C00F018FD2B68013BA8
:1012200006E00748211C00F011FD2B681C700133FB
:101230002B6038BDC0020010EF400000B901001063
:10124000FE40000008B503E000F0A0FBFFF7C4FF7C
:1012500000F0BEFB0028F7D108BD000008B5034A26
:10126000034B04481A6000F0F1FC08BDB9010010FE
:10127000C0020010F2400000044B40211A680A43EB
:101280001A60034B01221A707047C04680800440E8
:10129000C802001070B50E4B061C1B780D1C141CE8
:1012A000002B01D1FFF7E8FF013E022E03D8094BC6
:1012B000B600F35800E0084B1A68012C03D1AC408B
:1012C00014431C6003E00124AC40A2431A6070BDCB
:1012D000C8020010804100000080005038B50F4B5C
:1012E000051C1B780C1C002B01D1FFF7C5FF00204B
:1012F000032D11D8281C012302F0E4FA0204060889
:10130000074A04E0074A02E0074A00E0074A10687B
:10131000A3401840431E984138BDC046C802001083
:10132000FC3F0050FC3F0150FC3F0250FC3F03508B
:1013300070B50E4B061C1B780D1C141C002B01D124
:10134000FFF79AFF013E022E03D8094BB600F3586F
:1013500000E0084B1A68012C03D1AC4014431C6018
:1013600003E00124AC40A2431A6070BDC802001023
:101370008C410000FC3F005038B5084B041C1B7822
:101380000D1C002B01D1FFF777FF23681822934330
:10139000236023681D43256038BDC046C802001085
:1013A0001F234209184001238340181C014B92005F
:1013B000D050704700E100E01F234209184001238C
:1013C0008340181C2032024B9200D0507047C04618
:1013D00000E100E0054B3F221A60054B01221A6034
:1013E000044B40211A688A431A60704724800440E5
:1013F000D88004403882044008B5044B40211A6864
:101400008A431A60FFF7E6FF08BDC04638820440F1
:1014100008B5154B1868FFF78DFD0720FFF7CCFFC7
:101420000820FFF7C9FF0A20FFF7C6FF0C20FFF7CF
:10143000C3FF0B20FFF7C0FF0920FFF7BDFF0B4ADA
:101440000023136001210A4A49421160094A1360CE
:10145000094A1360094B01221A60094B1A680132CC
:101460001A60C04608BDC04608000010048204404F
:101470000882044004C000403CC0004000C000405E
:10148000CC02001008B5FFF72BFC0A480021FFF73B
:1014900073FF09480021FFF76FFF08480021FFF79D
:1014A0006BFF07480021FFF767FF06480021FFF7A1
:1014B00063FF08BD0840044000400440AC400440C5
:1014C000144004401C400440F8B5071C0C1C72B6C4
:1014D000FFF7D8FF434B1A68434B1A60002F01D027
:1014E000424B00E0424B434A04211360424B434DC0
:1014F0001A680A431A6000232B609C4218D0072008
:10150000FFF74EFF0820FFF74BFF0A20FFF748FFC9
:101510000C20FFF745FF0B20FFF742FF384B394AFD
:1015200019680A401A602A68EC235B0113432B6098
:10153000002F4FD0344B354C354900260E60201C0F
:101540001E60311CFFF718FF301C0921321CFFF709
:10155000A1FE301C0921321CFFF7EAFE2D4B802230
:10156000196811431960236807218B43236023689E
:1015700002210B4323607B00DB1999015B189B0060
:101580002549DF19254B0F6003211960244B25499C
:10159000186801401960196809200A431A60FFF7AA
:1015A000FFFE174A802311689B00194311602A68C7
:1015B000022113431C4A2B60012313601B4A116054
:1015C0001B4A134913601660136010681842FCD060
:1015D00001230B60174B012252421A6062B630BFE2
:1015E000F8BDC0463882044034820440BF18000071
:1015F000FF1800003082044010ED00E00482044037
:10160000008204407FE2FFFF044001406440044048
:1016100004C000408080044018C0004014C0004056
:101620003CC000400FF0FFFF788004407080044011
:10163000748004400882044008B5FFF745FF08BDE8
:1016400000B5064B1A6801321A601B68013303D1DA
:10165000034B1A6801321A6000BDC046D402001064
:10166000D002001000B5074B98420AD8064A002362
:101670001360064A01381060054A1360054B0722C3
:101680001A6000BDFFFFFF00D402001014E000E06C
:1016900018E000E010E000E000B50C4A13680028F4
:1016A00000D10120C1438B4204D809E01168814276
:1016B000FCD301E0591C081811689942F6D203E0E6
:1016C0001168C91A8142FBD300BDC046D402001084
:1016D00010B5064BFA211868054B89001C6802F00A
:1016E00005F9044B5C43201810BDC046D40200101D
:1016F000D002001037894100034B01221A60034BCE
:101700001A6801321A60704700C00040D802001009
:10171000034B01221A60034B1A6801321A607047AA
:1017200000000140DC020010034B01221A60034B51
:101730001A6801321A60704700400140E002001050
:10174000034B01221A60034B1A6801321A6070477A
:1017500000800140E402001000B5002803D1044BD2
:1017600001221A6003E0012801D1024B186000BD7C
:10177000044001400480014000B5002802D1044B20
:10178000186004E0012802D1024B00221A6000BD5B
:10179000044001400480014010B500280FD1124BD5
:1017A00080221C68920022431A60104B03221860AA
:1017B0000F4B19600F4B1A608022D20211E00128F2
:1017C00011D1094B80221868D20002431A600A4BDB
:1017D00000221A60094B03221960094B1A6080220B
:1017E0001203084B1A6010BD80800440E002001014
:1017F0001840014014400140E402001018800140EC
:101800001480014000E100E008B5184B1A680E236F
:101810001340062B0DD1164B9E221B68DBB21342E0
:1018200004D0144A5360144B1B681EE0D9071CD522
:1018300001E0042B05D1104B1868C0B200F0B7F8D6
:1018400013E00C2B06D10B4B8022596852000A433F
:101850005A600AE0022B08D1054B1A68054B910625
:1018600001D5002200E001229A6008BD08800040F6
:1018700014800040E80200100080004000487047DB
:10188000E802001070B52A4C2A4B80229203DA67D6
:1018900000219022061C201C00F010FA0023A360F7
:1018A00000F06EF8244B07251A68244CAA431A60EE
:1018B0001968012211431960214B1968A943196065
:1018C0001968114319601F4B8021186849010143B1
:1018D00019601D4B1A608322226019681B4B18681F
:1018E00002F004F8311C000902F000F81849030A5C
:1018F000184A0B60C0B2032310602360164B1D60B2
:10190000164B186860201C680440602CFBD101E075
:10191000146800E001201C680442F9D1044B012244
:101920001A700F4B802292031A6005230B6070BD62
:10193000E802001004E100E0A44004400C800040F4
:10194000A84004408080044098800440B404001003
:101950000480004000800040088000401480004067
:1019600000E100E000B5044A202311681942FCD0D0
:10197000024B186000BDC04614800040008000404B
:1019800008B5FFF77BFF0023437308BD08B5FFF7D9
:1019900075FFC27B031C8218107CDA7B7F21013229
:1019A0000A40DA735A7B013AD2B25A7308BD10B5B5
:1019B000041CFFF763FF837B7F22C3181C74837BA7
:1019C000013313408373437B0133DBB2437310BD98
:1019D00008B5FFF753FF407B431E984108BD30B563
:1019E000002402E00570013401301D5D002DF9D1A5
:1019F000121B131C02E00170013B0130002BFADCCA
:101A0000D043C0170240A01830BDF8B5051C0F1C0C
:101A10001E1C541E092B01D800240FE0181C0A219B
:101A200001F064FF221C031C391C281CFFF7EDFF8A
:101A3000041C2D1805E02F7001340135013A002AED
:101A4000F9DC301C0A2101F095FF30312970601C4F
:101A5000F8BDF8B50C1CD9175F18061C4F40551E71
:101A6000092F12D9381C0A21002B03DA01F03EFF9E
:101A7000434202E001F03AFF031C211C2A1C301CE7
:101A8000FFF7E7FF041C351813E0002B00DA951E62
:101A9000002201E0B4540132A91A0029FADCEC4317
:101AA000E4172C403519002B03DA2D232B70013459
:101AB0000135381C0A2101F05DFF30312970601CAE
:101AC000F8BD73B5069E041C1D1C3009531E00286A
:101AD0000AD000901A1C201C2B1CFFF7F2FF2418C0
:101AE00005E0217001300134013A002AF9DC0F23AE
:101AF0001E40092E01D8303604E0002D01D03736C3
:101B000000E057362670013076BDF0B585B0041C74
:101B10000F1C002801D00021017000256BE0252951
:101B200003D021700132013405E05178252904D118
:101B300021700232013401355DE0302903D00132D9
:101B40000292202101E002320292029E9C463278EB
:101B50002D3A50424241B6180296002205E00A236F
:101B60005A438218303AD2B201363078031C303BE7
:101B7000092BF4D90296AE186346BE4201D97A1BEE
:101B8000D2B269280ED006D863282CD0642809D098
:101B900058283ED119E075280AD078280FD073282C
:101BA00037D11AE01E1D201C1B68FFF752FF04E00E
:101BB0001E1D201C1B68FFF728FF331C17E01E1D8D
:101BC0001B68201C0093002304E01E1D1B68201CC2
:101BD00000930123FFF775FFEFE71E1D201C1B6814
:101BE000FFF7FDFEE9E71A68012022700433029A2C
:101BF000241801322D181178BD4201D200298ED14E
:101C00000023BD4201D2237005E0013C2370013D59
:101C100001E001256D4205B0281CF0BD10B50C1C7B
:101C2000131C6421221CFFF770FF10BD00B5031CBC
:101C30009BB00A1C01A8191CFFF7F0FF632800DD08
:101C4000FEE701A800F0A6F81BB000BD0FB407B571
:101C500004A901C90191FFF7E9FF03B008BC04B072
:101C600018470EB403B503AA02CA0192FFF7D6FFC4
:101C700002B008BC03B0184770B50323041C184217
:101C800005D10D1C041C194201D1934201D300233C
:101C900011E0131C40CD043B40C4032BFAD8141FA1
:101CA000A4080134A400032309191A400419EEE71B
:101CB000CD5CE55401339342FAD170BD30B50B04CD
:101CC0000D061D430D430B021D430323041C9342C9
:101CD0000DD218420BD1131C043B20C4032BFBD89C
:101CE000141FA4080134A40003231A40041900237C
:101CF00001E0E15401339342FBD130BD00B5002334
:101D000000E00133C25C002AFBD1181C00BD00B505
:101D1000031C01E0013101330A781A70002AF9D15D
:101D200000BD30B5031C002406E01D5D085D281AC7
:101D300005D10134002D02D09442F6D1002030BDEF
:101D400000B502E00130002B06D00A78037801319B
:101D50009342F7D0981A00E0181C00BD08B5FFF7B1
:101D60004DF90B4BFA211868890001F00DFEFFF7C1
:101D700079FCFFF781FAFFF73FFB96200002FFF79F
:101D800081FDFEF747FEFEF733FEFFF767FA08BD59
:101D9000B404001010B5041C02E00134FFF7E2FDAA
:101DA00020780028F9D110BD30B5F8238A01DB0076
:101DB00013404A05920E1343F822120211401943B0
:101DC0000A235943CA1083181C1CEB345D7824780D
:101DD000EA336C401B7824021C43835C201C58406F
:101DE0000723194008418005800D30BD08B5054B1B
:101DF000011C984201DD044BC1180448EA38FFF782
:101E0000D3FF08BDFF17000000F8FFFF9841000056
:101E100008B54018511A013101F018FE08BD08B587
:101E2000801889189A1A0132FFF726FF08BD0000B2
:101E300010B5CB00591A074B0F22C9180023CC5CF0
:101E400014400470CC5C0133240944700230072B29
:101E5000F5D110BD5405001010B5CB00591A064B32
:101E6000C91800234278047812012243CA5401336E
:101E70000230072BF6D110BD5405001030B5B14B20
:101E800087B0D96EB04D4A1E91416A46D175A96A94
:101E90001A1CC806400F0138062807D801F012FDA9
:101EA000040C1F1217191C00022409E05A6E163286
:101EB0009200D3581C1C15E05B6E16339B00D4585F
:101EC00000230FE09B6DD46DA3420ADC0AE00224DC
:101ED00003E00C24032305E00D24231C02E00D2461
:101EE000EEE70D242C6148111F2800D922E16A4633
:101EF0001732944901F0F0FC2000220028002A004B
:101F00002D002F00380040004400490051005F00C0
:101F100067006F00770085009300A200B400C30043
:101F2000D500D300E300E600E900F100010105015E
:101F30000F01110113011901081C00E08348191C4D
:101F4000221CFFF765FFF5E08148F8E70A1C0E3216
:101F500003E07E4809E00A1C1C32081C111C1A1CF4
:101F6000231C01F0F9F8E5E07948011C0E391A1C30
:101F7000231CFFF754FFDDE07448011C0E31EEE72F
:101F80000A1C1C32081C111CF1E70A6E1020002AE2
:101F900000D00A200A1C0E3206E00A6E1020002A29
:101FA00000D00A200A1C1C3200946C4617340290A0
:101FB0000194081C51E001201070086E10220028C6
:101FC00044D00A2242E00A6E1020002A00D00A20E3
:101FD0000A1C0E320EE001201070086E102200283C
:101FE00055D00A2253E00A6E1020002A00D00A20A1
:101FF0000A1C1C3200946C46173402900194081C91
:1020000078E00A6E1021002A00D00A21504A684662
:102010001730019002910094101C111C1DE00A6EF3
:102020001020002A00D00A20494A00946C46111C56
:10203000173402901C390194101C0EE0096E012027
:1020400010701022002900D00A224149684617303A
:10205000019002920094081C002201F087F869E0C8
:102060000A6E1020002A00D00A20394A00946C46DB
:10207000111C173402901C390194101C3AE0096EAF
:10208000012010701022002900D00A223049684631
:102090001730019002920094081C00222AE00120CF
:1020A00010700A6E1021002A00D00A21284A6846C2
:1020B0001730019002910094101C00211AE0009248
:1020C00022481CE00092224819E00A6E1020002AE3
:1020D00000D00A200A1C1C3206E00A6E1020002ADA
:1020E00000D00A200A1C0E3200946C46173402906D
:1020F0000194002001F063F81CE00092081C00210C
:1021000004E00D1C1C35081C0092291C1A1C231C01
:1021100001F0B0F80EE0081C02E00C4800E00C48AA
:10212000191C221C01F0BFF804E0081C221C191C19
:1021300001F0C4F86B46DA7D024B07B00120DA6685
:1021400030BDC046B8040010540C0010C604001086
:10215000D404001010B506490B1C88331A68141CEF
:102160001E34A4006050013203210A401A6010BDE1
:10217000B8040010054B0320191C88310A68013A85
:1021800002400A601E329200D0587047B804001016
:10219000F8B5114D2C1C8C3420680130FFF726FE59
:1021A0000E4B0122D8629F6AAB6E061C02409A4217
:1021B00010D1830703D420680230FFF7CBFFFF2341
:1021C0009B001E40B601BF10044B8C3537430122E3
:1021D0002F60DA600220F8BDB8040010540C001023
:1021E00030B50C4B0C489A6A031C8C331C68D30521
:1021F0009B0E910500D5403B856E921001210A404F
:10220000AA4204D1E3188C300360024BD96001204C
:1022100030BDC046540C0010B804001008B5084B7F
:102220005A1CD07F9A1CD27F000112021043DA7F21
:102230000333DB7F10431B031843FFF78BFF08BDFD
:10224000B804001038B5FFF795FF064903230F22A5
:10225000051C5C181540013325770011072BF7D1B9
:1022600038BDC046B804001008B5FFF783FF034B24
:1022700001228C331860024BDA6008BDB8040010EC
:10228000540C001010B5064CA36E002B06D0FFF7BF
:1022900071FF044B8C3401222060DA6010BDC0460F
:1022A000B8040010540C001010B5064CA36E002B9F
:1022B00006D1FFF75FFF044B8C3401222060DA6007
:1022C00010BDC046B8040010540C001008B5124BE5
:1022D0001B68002B00D09847104B5A69002A15DD67
:1022E000012A07D1DA69002A04D09A610022DA6152
:1022F0000A225A615B690322191C91430A1E02D00B
:10230000074A0121D166054A013B5361044B9033D2
:102310001A68024B5A6208BD78030010540C001072
:10232000B804001000B5064B5A69002A07DD9A6907
:102330000F21044B1140D97712110133DA7700BD18
:10234000540C0010B8040010044B597F9A7F090107
:1023500012020A43197F0A435A677047B8040010F3
:1023600030B50B1C093B012B0FD8084A00239C18E1
:10237000257FC45CA54205D0054B08395A68114336
:10238000596002E001330E2BF1D130BDB8040010CA
:10239000540C001008B50E4B1B68292B17D00829C8
:1023A0000DD0192913D1427808231A4202D00022F5
:1023B000027002E00F2303700723437005E000233F
:1023C0001A1CC25401330E2BFBD1FFF745FD08BD8B
:1023D000540C00101FB50D4B5C6F002802D00F226B
:1023E000944304435C676846211CFFF721FD68465F
:1023F000211CFFF7CFFF054A00236C46185D991892
:10240000013308770E2BF8D11FBDC046B804001069
:102410001FB5124B0F225C6F944304435C67104B53
:102420001B68292B01D0082C17D06846211CFFF708
:10243000FFFC6846211CFFF793FF084A0023991808
:10244000097F6846195401330E2BF8D1211CFFF780
:10245000A1FF6846211CFFF7FFFC1FBDB804001058
:10246000540C00101FB5114B114C1B68292B02D0C6
:10247000636F082B18D0616F6846FFF7D9FC616F56
:102480006846FFF76DFF0A4C00231A19127F694650
:102490005A5401330E2BF8D1616F6846FFF77AFF6B
:1024A000616F6846FFF7D8FC1FBDC046540C001092
:1024B000B804001010B50D4C631CD87FA31CDB7F43
:1024C00000011B021843E37F1843E31CDB7F1B035F
:1024D0001843FFF78BFC0F23021C1A4022770211CE
:1024E000134000126377A07710BDC046B8040010F7
:1024F000044B5A6E16329200D258121A51424A4177
:10250000DA667047B804001000B5064B5A6E1632F2
:102510009200D1580139D150002901DA0D21D15052
:1025200000BDC046B804001000B5064B5A6E163206
:102530009200D1580131D1500E2901D10021D15042
:1025400000BDC046B804001000B5094B5A6E1632E3
:102550009200D2580D2A03D11A1C2932127805E0B4
:102560009A18507F117F0001021C0A435A6500BD72
:10257000B804001010B5084B0F245A6E16329200A2
:10258000D1585A6D58181440013104770D2902DCD6
:102590005B1812111A7710BDB804001030B50F4B3C
:1025A0005A6E596D16329200D2580D2A07D11C1C52
:1025B00029342478F02008402043586507E0981813
:1025C000447F057F24012C435C650B114377034B4B
:1025D0009A180F231940117730BDC046B804001077
:1025E00008B504480022011C1C390D23FFF717FC15
:1025F00008BDC046F004001008B504480022011CC4
:102600001C310D23FFF70BFC08BDC046D40400109D
:1026100008B504480022011C1C310D2300F09CFD6C
:1026200008BDC046D404001008B504480022011CAF
:102630000E390D23FFF7F3FB08BDC046E20400107E
:1026400008B504480022011C0E310D23FFF7E7FBFB
:1026500008BDC046D404001008B504480022011C7F
:102660000E310D2300F078FD08BDC046D4040010E3
:102670000C4A0023111C46310B70111C47310B70A2
:10268000111C48310B70111C49310B70111C4A315F
:102690000B70111C4B310B70111C4C314D320B70F7
:1026A00013707047B804001000B5074A011C0423DA
:1026B00000208A1804E0D118463109784000084308
:1026C000013BF8D200BDC046B804001030B5074A3F
:1026D00000238918012206E0CC18051C4634154059
:1026E000257040100133042BF6D130BDB804001022
:1026F00038B50020FFF7D8FF084C051C0021207FCB
:10270000FFF7E4FF25770420FFF7CEFF0421051C27
:10271000607FFFF7DBFF657738BDC046B804001067
:1027200010B50020FFF7C0FF034C20770420FFF70F
:10273000BBFF607710BDC046B804001010B5054C53
:102740000021207FFFF7C2FF607F0421FFF7BEFF5B
:1027500010BDC046B804001010B5094C231C8C33C2
:1027600018680130FFF742FB064B021CD8620F23AA
:102770001A4022770211134000126377A07710BD30
:10278000B8040010540C001010B5094C0021201C96
:102790000D22FFF73DFB201C0E3000210D22FFF71C
:1027A00037FB201C1C3000210D22FFF731FB10BD30
:1027B000B804001010B50C4B00211A1C187F1C78AF
:1027C00001312043187701330E29F7D1936E002B86
:1027D00008D0064B1B690D2B04D1137F111C293126
:1027E0000B70537310BDC046B8040010540C001099
:1027F00010B50C4B00211A1C1C7F187801312040A9
:10280000187701330E29F7D1936E002B08D0064BB1
:102810001B690D2B04D1137F111C29310B705373CD
:1028200010BDC046B8040010540C00107FB5002342
:102830000C4A0D251C1C1118097F01306E46995554
:10284000C60F8542664176420133111C30400E2B83
:10285000F1D100236C46185DCA18013310770E2B96
:10286000F8D17FBDB804001010B5074B5A6E163270
:102870009200D1585C1801392077D150002901DA33
:102880000D21D15010BDC046B8040010034A0023EA
:10289000111C943198320B6013607047B80400101B
:1028A000034B012194331A684A401A607047C046AE
:1028B000B8040010044A002313678C321360034BE2
:1028C0000122DA607047C046B8040010540C0010B2
:1028D00008B59A4B0F20996A994A8B1018408911B4
:1028E000013852560E2800D9C1E000F0EBFF081164
:1028F0001A2327C02EC0C037C0C0C03B3F00002AEB
:1029000000DAB4E08F4B9A18403200239371A9E0AB
:10291000002A00DAABE08B4B01209A18403290710C
:10292000A4E0002A00DAA2E0864B9A18403292799D
:10293000DA6697E0081CFFF797FF93E0002A00DAB9
:1029400095E0101CFFF7D4FD8CE0002A00DA8EE041
:102950007C4B596E16318900CA5083E0081CFFF782
:1029600057FD7FE0081CFFF735FD7BE0002A00DA09
:102970007DE0101CFFF75AFF74E0724B0120983382
:10298000186073E0FFF7E0FD6CE0FFF793FF69E08C
:10299000FFF726FE66E0FFF7EDFD63E0694B0022DE
:1029A0005A665FE0FFF728FE5CE0FFF7F7FD59E0AD
:1029B000644B0120586659E0FFF72AFE52E0FFF70A
:1029C000CBFE022052E0FFF72FFE4BE0FFF726FC84
:1029D00048E0FFF735FE45E0FFF7D6FE42E0FFF79F
:1029E00031FC3FE0FFF738FE3CE0FFF79BFC39E0AD
:1029F000544B00221A6635E0FFF7A6FC32E0514B3B
:102A00000120186632E0FFF741FF2BE0FFF72AFDB7
:102A100028E0FFF745FF25E0FFF74CFD22E0FFF738
:102A20008DFE1FE0FFF72EFC1CE0FFF7C3FE19E050
:102A3000FFF776FE16E0FFF737FC13E0FFF7D8FE4E
:102A400010E0FFF715FE0DE0FFF740FC0AE0FFF78E
:102A50005BFD07E0FFF74CFE04E0FFF765FD01E0DA
:102A6000FFF702FC012001E00120404208BD982B45
:102A7000BED03EDC382B9BD01DDC1C2B00D187E761
:102A80000CDC0C2B00D178E702DC002BEAD0EBE762
:102A9000162B00D176E7182BE6D176E7282B00D14C
:102AA0007CE702DC262BDFD175E72C2B00D179E700
:102AB000362BD9D179E7662B00D18AE70CDC4C2B79
:102AC00000D17CE702DC3C2BCED175E7562B00D140
:102AD00079E75C2BC8D179E76C2B00D17FE702DC6A
:102AE000682BC1D178E7762B00D17BE7882BBBD14F
:102AF0007BE7E62B00D19BE726DCC82B00D188E7DB
:102B00000CDCA82B00D17AE702DC9C2BACD173E75C
:102B1000B82B00D177E7BC2BA6D177E7D62B00D115
:102B20007DE703DCCC2B00D09EE775E7D82B00D1E6
:102B300078E7DC2B00D097E777E7C046540C00100D
:102B4000987D0000B8040010F32B00D17CE70EDC68
:102B5000EC2B00D172E703DCE82B00D084E76AE7B6
:102B6000F12B00D16DE7F22B00D07DE77AE7F62B51
:102B700000D16FE703DCF52B00D075E767E7F72B93
:102B800000D16AE7F82B00D06EE769E738B5184C3A
:102B9000231C8C331868FFF729F9E26E154BA266E7
:102BA0000022E266DA6003229862251C10401C1C99
:102BB000022809D090420AD0012802D0FFF788FEEF
:102BC00007E0FFF7E5FA04E0FFF758F901E0FFF747
:102BD00007FB002807DDE368002B04D12B1C8C3396
:102BE0001A6812181A6090352B681B182B6038BDB4
:102BF000B8040010540C0010034B0122DA660F22B7
:102C00009A775A771A777047B804001010B5054CB8
:102C10000549201C00F01AFFFFF7EEFF0123636651
:102C200010BDC046B80400109C07000000B5074B5B
:102C300000201B680F2B08D1054B1A78824204D163
:102C40001868044B1840431E984100BD84000010D2
:102C5000B804001000FFFF0038B5164B1A1C98325C
:102C60001268002A04D0144B1D6801231D4001E0A6
:102C700094331D68114CA3689D4202D16268002AFA
:102C800016D0002D02D1002B0AD111E00C4B1B688D
:102C9000002B02D06168281C98470023636006E07F
:102CA000074B1B68002B02D0281C291C9847A560E5
:102CB00038BDC046B804001098030010540C001032
:102CC0009003001013B5002300930193244B1B685D
:102CD000002B02D0684601A998472249009B08783A
:102CE000214A00280CD0002B02D00223137035E0BB
:102CF0001378013BDBB21370002B2FD10B7009E06E
:102D0000002B0CD11378002B28D0013BDBB21370C1
:102D1000002B23D1154A1360154A13601EE0144995
:102D20000968581A444260414000107011484469D3
:102D3000021C002C04D08B4202D10A2343610DE017
:102D400000290BD10A21516101999361D161084A8F
:102D50001360064B02221960034B1A7013BDC04664
:102D6000800300109C03001084030010880C0010E6
:102D7000840C0010540C001008B5FFF7A3FF08BD29
:102D800010B5094C20600948016009490A60094AE8
:102D90001360094B029A1A60084B039A1A60084A9A
:102DA000084B1A6010BDC04690030010800300104D
:102DB0008C030010880300107C03001084000010B6
:102DC000792D00007803001008B5084B084A1968EF
:102DD00012688A1A1A6006D5FA2252001A60054B48
:102DE0001A6801321A60FFF737FF08BD880000102B
:102DF0007C03001098030010F7B50E1C0E21051C73
:102E0000019200F023FE1A4B03240C279E420FDD93
:102E100009236B7301232B7328E0301C0A2100F077
:102E200009FE301C29550A2100F0AEFD0134061CB4
:102E3000002E06D0E30F0022A7425341DBB293429B
:102E4000EBD1019AA31A033B2B70621B2B1C01E0F0
:102E5000195D5973013BD1180229F9D10F231C1BAD
:102E6000002301E0013C2B55032CFBDCF7BDC046E1
:102E7000FFC99A3B38B50C4B01221A700B4B02224A
:102E80001A700B4D0B4C08E01868884208D01B687C
:102E90002360FFF799FFFFF715FF2B682168024AAF
:102EA00010780028F0D138BD9C0300108403001076
:102EB0008803001094030010F7B51C4D9B235B00A2
:102EC0000E1C1B4AE95C1B4BAC5CEB5C002902D07E
:102ED0000F22144002E08021072449009A22520068
:102EE000AF5C154ACB1AAA5C3435BA1A80277F002A
:102EF000791A009107210C1B013210490194FEF749
:102F0000B0FE00230E4F33704124FF35301CFEF716
:102F1000F5FE2A786B783018D31A391C221C01343C
:102F2000FEF79FFE013D462CF0D1F7BDB80400101E
:102F3000370100002F01000035010000A87D0000CE
:102F4000B57D000070B5434B434C1A1C9432126897
:102F500090B0A061E161002A17D118280BD1C329D4
:102F600009D13E4A12680F2A05D1181C38300E21AB
:102F7000162200F0DDF8A369182B04D1E369332B86
:102F800001D100F07FF8FFF737FE0A23314D63616E
:102F9000334E01232B678C35FFF7F8FD2B68B342C6
:102FA00016D006DC2F4A93420DD02F4A93423AD1D5
:102FB0001DE02E4A934210D02D4A934220D02D4A34
:102FC000934230D10EE0254B1B680A2B2BD112E027
:102FD000224B1B680B2B26D10DE0204B1B680C2BC2
:102FE00021D108E01D4B1B680F2B1CD103E01B4BAC
:102FF0001B68102B17D1FFF72FFEFDF768F812E0C2
:10300000164B1B680F2B0ED11B4C2368002B0AD0CC
:10301000684608A9FFF750FF2368684608A9984743
:103020002B6827332B60154B1A68154B10681968ED
:10303000884205D012681A60FFF7C6FEFFF742FE0D
:10304000044B1B6F002BA7D1FFF706FEFFF712FF03
:1030500010B070BDB8040010540C001084000010B3
:10306000130D0000070C00006A0C0000990D000011
:103070003E270000790D00008C030010880300102B
:103080009403001070B5254C23681D68FFF7F2FE0D
:1030900023681A689542FCD01E68FFF7ADFD204BEF
:1030A0000A22204C5A6118229A611522DA61231CE7
:1030B000903300221A60FFF79FFD2D36012323670E
:1030C000FF36164C184D0AE0FFF760FD23682A68AA
:1030D0001968914203D01B682B60FFF775FE2368C7
:1030E0001B689E42F0D10F4C1820231C9033002106
:1030F0001D68FFF727FF0D4B281C196800F044FCE2
:103100003834011C0422201CFFF776FE044B1822E1
:103110009A610022281CDA6170BDC0468803001045
:10312000540C0010B8040010940300107C0300102D
:10313000F0B501240DE005780B1C254006E0C65CC7
:10314000ED0077083D43C554351C2540013BF6D5BD
:10315000013A002AEFDCF0BD30B504E0845C8D5C00
:1031600085548C5401329A42F8DD30BDF7B5099D83
:103170000AAC2678089F2C7894461D1C002A0DD195
:1031800018E063465B5D4A5DD21813190192002472
:10319000B34201DB9B1B012443550135BD42F0DDE9
:1031A0000AE0CA5C12190024B24201DB921B01241E
:1031B000C2540133BB42F4DD099B1C70F7BDF7B567
:1031C000099E0AAC2778089D347800282FD0002962
:1031D0002AD01E1C9446002A0ED1013F18E06346F7
:1031E0009B5D8A5DD21A131B00240192A34201DA6F
:1031F000DB19012483550136AE42F0DD37E0CA5CAD
:10320000121B0024561C01D13A1C0124C254013364
:10321000AB42F4DD2BE0D15C49420C1B211E01D0F6
:10322000E1190124C1540133AB42F4DD1FE0002950
:103230001BD0181C002A06D10EE00E5C135C013076
:10324000F31A1C1BE40FA842F7DD10E0CA5C01333F
:10325000141B013462425441AB42F7DD07E0D15CFC
:10326000013349420C1B611E8C41AB42F7DD099AC8
:103270001470F7BD70B5049D01242C70141C002936
:1032800005D10BE0065D0A5D96420BD101349C42EC
:10329000F8DD05E0815C002904D101329A42F9DDB4
:1032A00000232B7070BD00B503E043185B784354D6
:1032B00001319142F9DB0023435400BD00B504E025
:1032C0008318013B1B788354013A8A42F8DC0023BF
:1032D000835400BDF0B5114B1A785B78825C1A40BC
:1032E00000D040220E4C0F49231C261C04C32C3650
:1032F00000221A6001240A1C123117785578C75D24
:103300003D4202D01F6827431F60023264008A4298
:10331000F3D10433B342EBD10020F0BD81010010A2
:103320001C0E0010CD00001030B512234B43334A61
:103330000131D3188A0051181A785C78825C1442E3
:1033400004D02F4A5F245218947054709A78DC7815
:10335000825C144204D02A4A7C24521853321470DE
:103360001A795C79825C144204D0254A7C24521874
:10337000A33214709A79DC79825C144207D0204C15
:103380005F226418251CA235A1342A7022701A7A93
:103390005C7A825C144204D0194A7C245218A03210
:1033A00014709A7ADC7A825C144204D0144A7C2429
:1033B0005218503214701A7B5C7B825C144207D026
:1033C0000F4C5F226418251C523551342A7022702C
:1033D0009A7BDC7B825C144204D0094A2E2452186A
:1033E000A43214701A7C5B7C825C134204D0044BC0
:1033F0005918F43127230B70002030BDCD00001088
:103400008C0C0010F8B52D4C071C0025201C202129
:103410004F22FEF753FC002D04D0221C7C233932AE
:1034200023701370231C4F33002101351970503461
:10343000052DEBD1214B2D22181C38300270181CA1
:1034400037300270A1209A705A7040005F221A54DF
:103450001B481A54A320400019541A490878497887
:10346000385C014204D0191C533152330A701A706F
:103470000024211C381C0134FFF756FF0A2CF8D118
:10348000114D124E00242B786A78FB5C1A4201D051
:10349000315905E03059FEF731FC0D49091A0A315E
:1034A0000C48043400F0DCFA0235242CEBD10A4934
:1034B000084800F0D5FA0520F8BDC0468C0C001075
:1034C00041010000810100108C000010A0000010DC
:1034D00083010010CC0D0010BD7D0000F0B585B05B
:1034E00001900027FDF784FA6A4C3E1C6A4A754237
:1034F000754113687D19012B05D168480D210C22F7
:10350000FDF714FB02E0002B00D1CDE0002303AA5D
:10351000537023687F210B405C2B00D198E02ADC9C
:10352000382B00D18EE013DC072B6AD006DC022B8F
:1035300000D193E0062B00D0B6E041E0212B00D172
:1035400084E0232B00D187E01C2B00D0ACE081E08D
:103550004F2B4ED007DC3F2B62D0402B62D0392B53
:1035600000D0A1E064E0542B76D05B2B3FD0502BF1
:1035700000D099E06AE0732B66D010DC662B3AD05D
:1035800005DC5E2B56D0622B00D08DE062E06F2B05
:103590003BD0712B52D06D2B00D085E02DE0792BE4
:1035A0004AD006DC762B4BD0772B3DD0742B7BD1C9
:1035B00046E07D2B23D07F2B25D07C2B74D135E0AA
:1035C00031231370022E4BDD231C083B1B6819406E
:1035D000542908D0032E43D0231C0C3B1A687F23A8
:1035E0001340542B3CD14C2203AB1A7038E03223E9
:1035F00035E0332333E0342331E035232FE0362325
:103600002DE037232BE0382329E039231370062ED1
:1036100026DD231F1B6819404723232920D11EE0E4
:1036200030231CE02D231AE0412318E0422316E04A
:10363000432314E0442312E0452310E046230EE028
:1036400048230CE04C230AE0502308E0522306E014
:103650004F2304E0552302E04E2300E0492313707A
:10366000ADB203A8291C0022FDF7D6FA23681A067A
:1036700005D5E91D89B20A480022FDF7CDFA236875
:10368000DA0572D50735A9B206480022FDF7C4FA5B
:103690006BE0C0461C0E001090010010553C00006D
:1036A0002A410000C57D000023680122134206D094
:1036B000A818C0B2002107220223FDF717FA2368D9
:1036C0000222134205D0A81DC0B200210623FDF737
:1036D0000DFA236804210B4205D0A81DC0B20222B6
:1036E0000623FDF703FA236808210B4205D0681C66
:1036F000C0B207220223FDF7F9F92368DA0606D5DE
:10370000681CC0B2042102220623FDF7EFF92368EA
:103710009A0606D5681CC0B2002102220623FDF7D6
:10372000E5F923685A0606D5681CC0B204210722B1
:103730000223FDF7DBF923681A0607D5281C093098
:103740000222C0B20821131CFDF7D0F92368DA0564
:103750000BD5EDB2281C0930C0B20B210A35FDF79C
:10376000AFF9E8B20A21FDF7ABF9013604340C37A2
:103770000B2E00D0BAE61B4803210622FDF7D6F92E
:10378000194D1A4E1A4F0024019A2B78D35C6A788F
:103790001A4205D0A3009859395D0922FDF73CFA79
:1037A00001340235092CEFD1FFF740FA002814D07C
:1037B00006240321201C00F0E7F80321C5B2201CD9
:1037C00000F038F9281CC9B2FDF77AF9092C01D1AB
:1037D0000B24EEE701340E2CEBDDFDF713F905B0F9
:1037E000F0BDC046923B00008C0000109401001018
:1037F000C400001070B5041CFFF76CFD201CFFF71F
:103800006DFE0A4B1B78002B0ED0201CFFF7FAFD33
:10381000074CC8235B00074EE518211C301C5034B0
:10382000FEF714FAAC42F8D1002070BD9D030010E1
:103830008C0C00106D3B000000B589B000280ED044
:10384000FDF7A1F801A80921FEF7F2FA6846123047
:103850000A21FEF7EDFA01A8FFF7CCFF08E0FDF71B
:103860009AF8044B1B78002B02D00348FEF7EEF9C0
:1038700009B000BD9D030010C77D000000B5FEE744
:1038800000B5FEE708B50A4B0A4A0B4903E0107879
:103890000132187001338B42F9D3084B08490022DA
:1038A00001E01A7001338B42FBD3FCF73BFEFEE7CD
:1038B00000000010207E0000B8010010B8010010C8
:1038C000480E001002B4714649084900095C4900DD
:1038D0008E4402BC7047C04603B47146490840009C
:1038E0004900095A49008E4403BC7047002934D06E
:1038F0000123002210B488422CD301242407A142C2
:1039000004D2814202D209011B01F8E7E400A1427E
:1039100004D2814202D249005B00F8E7884201D319
:10392000401A1A434C08A04202D3001B5C082243F1
:103930008C08A04202D3001B9C082243CC08A04262
:1039400002D3001BDC082243002803D01B0901D04E
:103950000909E3E7101C10BC7047002801D00020C3
:10396000C04307B4024802A14018029003BDC046FC
:10397000D90000000029F0D003B5FFF7B9FF0EBC55
:103980004243891A1847C046002941D010B4041C8C
:103990004C40A44601230022002900D549420028BA
:1039A00000D5404288422CD301242407A14204D2EE
:1039B000814202D209011B01F8E7E400A14204D2CE
:1039C000814202D249005B00F8E7884201D3401AE5
:1039D0001A434C08A04202D3001B5C0822438C0807
:1039E000A04202D3001B9C082243CC08A04202D371
:1039F000001BDC082243002803D01B0901D0090961
:103A0000E3E7101C6446002C00D5404210BC704710
:103A1000002806D003DB0020C043400801E08020DE
:103A2000000607B4024802A14018029003BDC04638
:103A3000190000000029EBD003B5FFF7A7FF0EBC6B
:103A40004243891A1847C0467047C04600B500294E
:103A500005D000230139037001300029FAD100BDDF
:103A6000F8B5041CA30719D1231C04CB0F4D104E2D
:103A700050199043021C201C32420FD1181C0B4FCE
:103A800004CBD5199543354208D1181C074F04CBF8
:103A9000D51995433542F1D000E001300378002B71
:103AA000FBD1FEF734F9201CF8BDC046FFFEFEFE38
:103AB000808080802578000D0A413A200020202552
:103AC000633A20000D0A4D3A20002020473A202575
:103AD0003032780D0A0053455249414C20434F4E35
:103AE000534F4C450025732072656164790D0A00BF
:103AF000444D313543435F4D454D3142000D0A423F
:103B000079652E2E2E0D0A004C43443A2530326939
:103B1000202D202569002573202573202025694D3F
:103B2000485A00563800202025692E253033695622
:103B3000004241543A2025696D560D0A000D0A25B0
:103B400030327820200057616974696E6720666F93
:103B50007220646174612E2E2E0D0A004261642071
:103B60006D6F64656C0D0A00526561642025730DEC
:103B70000A004F4B004641494C4544006F6E006FB0
:103B80006666004C43442064656275672025730DAA
:103B90000A00000000005C000C000C7C287C7C44C7
:103BA0007C241048285408000C0038440044380095
:103BB0002010081038108040001010100040002025
:103BC0001008384438007C006454484454281C10C1
:103BD0007C4C542438542004740C2854280854383D
:103BE0000050008050001028442828284428100441
:103BF0005408384C5C7814787C54283844447C440D
:103C0000387C54447C14043844347C107C007C00A0
:103C100020403C7C106C7C40407C087C7C047C7C9C
:103C2000447C7C14083844787C1468485424047C10
:103C3000047C407C3C403C7C207C6C106C1C601CF8
:103C400064544C7C4400081020447C000804088024
:103C500080800408000007080400000000BF01BFC6
:103C6000010905000007000700070007130A00000C
:103C70002000E400FC003F00E700FC003F002700BC
:103C8000040F0800000C011E01FF03FF032201E2E4
:103C900001C2190D00000E001F0011019101FF006B
:103CA0007E00FC00FE0113011101F001E0140A0086
:103CB00000EE00FF0111011101BF01EE00E0013033
:103CC000011001050300000F000F0A050000F800B5
:103CD000FE03070701040B060000000001040707AC
:103CE000FE03F80F08000000000A000E001F001F6E
:103CF000000E000A11090000100010001000FE0064
:103D0000FE0010001000100804000000048007806E
:103D1000030D07000010001000100010001000102C
:103D2000080400000000800180010D07000C000F56
:103D3000C003F0003C000F00030F080000FE00FF6E
:103D400001010101010101FF01FE10080000000056
:103D500002010201FF01FF01000100011008000043
:103D60008601C7016101210131011F010E010F0808
:103D7000000082008301110111011101FF01EE1108
:103D8000090000300038002C002600FF01FF012050
:103D900000200F08000080009F011F011101110188
:103DA000F101E10F080000FC00FE010B010901090F
:103DB00001F901F00F08000001000100C101F1014B
:103DC0003D000F00030F080000EE00FF011101117C
:103DD000011101FF01EE0F0800001E003F0121014B
:103DE0002101A101FF007E0804000000008C018C6D
:103DF000010804000000048C078C03120900002055
:103E00000070005000D80088008C010401040111EA
:103E100009000048004800480048004800480048A1
:103E2000004811090000040104018C018800D80039
:103E300050007000200D07000002000300B101B91E
:103E4000010F0006190D0000F800FC010603FB0637
:103E5000FD0505050505FD05FF050601FC01F81238
:103E60000900008001F0017C004F004F007C00F051
:103E70000180010F080000FF01FF01110111011F66
:103E800001FE01E0110900007C00FE008301010138
:103E90000101010183018211090000FF01FF0101FD
:103EA00001010101018301FE007C10080000FF01F7
:103EB000FF01110111011101110111010F08000091
:103EC000FF01FF0111001100110011000112090092
:103ED000007C00FE008301010121012101E301E2D8
:103EE0000112090000FF01FF011000100010001076
:103EF00000FF01FF010A0500000101FF01FF0101B0
:103F0000010B060001000101010101FF01FF100882
:103F10000000FF01FF0138006C00C60083010101B1
:103F200010080000FF01FF01000100010001000175
:103F30000001160B0000FF01FF010F003C00F00024
:103F4000F0003C000F00FF01FF0112090000FF011B
:103F5000FF010F001C007000E001FF01FF01130AC8
:103F600000007C00FE0083010101010101018301C9
:103F7000FE007C0F080000FF01FF0121002100214D
:103F8000003F001E140A00007C00FE0083010101B6
:103F9000010101038307FE047C0412090000FF01F4
:103FA000FF01210021007100DF008E0100011109D5
:103FB00000008E009F011101110111011101F30197
:103FC000E211090000010001000100FF01FF0101F1
:103FD00000010001110900007F00FF0080010001C5
:103FE00000018001FF007F1109000007001F007819
:103FF00000E001E00178001F0007190D00000F002C
:104000007F00F001E0017C001F001F007C00E00148
:10401000F0017F000F120900008301C7016C003816
:104020000038006C00C7018301110900000100077E
:10403000001E00F801F8011E00070001120900002F
:104040008101C1016101310119010D010701030164
:1040500000070008000A010018111013383130332E
:1040600078717073C8C1C0C388818083848487825B
:10407000C5C4C7C275747772353437321514171238
:1040800002070208020100030109030402040205F9
:10409000030500062024282C383C4044484C46693F
:1040A000726D776172652025735F56380D0A0025A1
:1040B0002D3130732025732573000D0A54797065F6
:1040C00020273C636F6D6D616E643E203F27206644
:1040D0006F7220706172616D730D0A0055707469A2
:1040E0006D65202575730D0A003F0025730D0A0DBF
:1040F0000A00564F5941474552203E3E2000256355
:104100000048656C70004E6F20706172616D7300C5
:104110004B6579207072657373003C6B6579313E35
:10412000203C6B6579323E202E2E2E0044756D703A
:10413000206D656D6F7279006C004C6F6164206D4D
:10414000656D6F7279007400546F67676C652064E9
:104150006973706C6179206F757470757420746FF9
:1041600020636F6E736F6C6500620052656164203E
:104170006261747465727920766F6C746167650032
:10418000008001500080025000800350FC3F01502D
:10419000FC3F0250FC3F0350CFB03C232324326C41
:1041A000D77C4099C8A6515E8DE53E70A3FB1A37B7
:1041B000737D74E4B2100AA3367ADB4E5C906155CD
:1041C000BD044BD57A775578106A346451A4FCABA2
:1041D000E8038A2CF3CE818F310DB2BF936D017845
:1041E00025854278870FA1136B63C0084BA61594F1
:1041F0006CDCECE894DA0CF9014492ED222532FBF8
:1042000064B2013886777059F33A04DA53543A921B
:1042100076022F3EAE196410DC7184F904D9D61CE5
:1042200079D1DC9B2794CA4246EC8ACDD7653F30D2
:104230002914769A5EAFDBE850FEB440676AF36BF0
:10424000EE1556ED356C833761BDB13AA3CC0178DC
:10425000296340AEAC5E14653F36B6DDFD9CE57269
:10426000DCEC52D195D845E6465B0CA07398106EF5
:10427000855684971F5D4DBE3ADCAC903A2670BEE1
:104280004DD58E2C8480ED200AEE1A7863EC89C619
:10429000C607917F8B5716AFBBC5325B1D9481E279
:1042A0000C5B7702594A1C20235108EC7A34F0E465
:1042B00063A2003AB43C88C0FE3BC9C06BA07C1A24
:1042C000A24D19D84B9C394F12437560D953A6C2E1
:1042D00078A07E65F90CE4DDFB522D2C17F3361027
:1042E00083A0D1DE0724D83A23E06D982274CE7ED5
:1042F00043A56BB528DE8660E45A8CE7738E2FA247
:10430000599D798F7EF5D0290E41C4E539B7D2C0C9
:10431000DFF884F79EFD3A9D7D1697A248FC628FD8
:1043200017EC3FA844CDFE02FCDAAC3551A824B608
:104330000C6EEC2734B042D8C69928346B37D98B31
:104340003C932573AFD1BD7C2578866CAA0B462D96
:10435000772066CB8C8BA7A012E2A454B5A54AEEB9
:104360004EAF3BB930FFDAA8C948D73D0F470885A3
:1043700039AD939E68149510C8468D2329719B53BF
:104380005689B1F5F9CA349B9872454463981C6B01
:1043900089433B6001F0BBB179F7921BB9F8BE3F8E
:1043A00030E8F78903E1A4CCA7442ED9D82DBF72F9
:1043B0001D42D87A25515A869BE5F42F63D6F49D89
:1043C000865ED66A1DDE6EA996B4C9A819CC15F111
:1043D000D610EFBEEB943360BCF6C9A4CC2F5D00C1
:1043E000C1B03E9881D73F8E2E9CE83D991B950128
:1043F00046733E9144592982E048A208A451A5245D
:10440000DB4D4D23CBEEA8629901AE0DF5AF79FDE2
:10441000E0890FC4C1254881058F5DA8709F8E611A
:10442000E8B5F9C9951F7E04554455B5E9E9EAE0B8
:10443000086AD440814C5F7C45BE640893C088986C
:1044400036F4A069E31A1925548EC423D6D788C33D
:104450009EA70D0FC71FEA993236024CB7ADC9D9D6
:10446000159AF35CFCE325DF976B5789B4BB6D0DA0
:1044700005DC8CAC2312356E7A599169C4FAF43A92
:104480009EFA71337E3A11F8AF2A170EF768E810DA
:10449000970297895A294E69AFF6E87928FE203F9E
:1044A0006A479F70685682C8C7B373B3046D950A94
:1044B00079F9D55A39E591E77B81DBC3D19E99B66D
:1044C000E51297A6A81AC4FCFDC26DDD6A02C4FA03
:1044D0008CBE3FE72D0CE81FF22BE2859CE58E8910
:1044E000AE5622C39946C8117A7ECB818A17BD3653
:1044F0002D1651504EB616536E9BB2099265E85672
:104500000A8B2C39E43B64678AFAB0F2D9F92EDEC3
:10451000CF5D996861E18E3964B01E2DD7D97414CE
:104520007A4C21FC8515D3F0E9929CDF988DC71A4F
:104530002DF71483B153048398131FA173BFD4596B
:104540001AF924735E7554A3FBD9AD797B47C4B7C0
:10455000AD6FD677586A3549E94C6CEA8CF6133A58
:10456000A33727035CE1CFEC91C897C8BDABBB96DE
:1045700013FEB61AD303F9AC0E14FF98746C7429A9
:10458000D359053DD7E1090E7F6256778DF6E7CA0C
:10459000F8A811E48AD8A542C6F7361944ECF5D537
:1045A000C2D725A2D300491C3C37DAC4E71A3DD94B
:1045B000FD99F64E1ECD52D164B8D5A3CC7F78D6E6
:1045C000B279C3E0138014D58FAEB270D8B19346E0
:1045D000EE8B2A33BE61097BADFADD9A5EDABDCB84
:1045E0008D516E7CA6D165ACE56EF2A3CA6545D649
:1045F000AA6E4D26E34D5FBB2CDECF4E8118BC71F9
:1046000052C838735A24102FEEE1FF4D27CC7E9C00
:104610008A9654BFCADBB3BD4585B6146F47B15304
:10462000D8D4175AE4F95E777407D742C4B344610B
:104630004CB7FAAD31369B5F96FB95D9EC01D1F2C0
:10464000FEF15390673902041386D63627E36E894C
:10465000CF5FF789E34E47CCCB542B4DEAE6939AD4
:10466000A0605E32A99405EC191F94A3F206DFE165
:10467000AA806D90D76EA88BE7027490757EA136E4
:104680003D45CC5066F3FD13298A0E386FD25F9EEC
:10469000B6DD2E4B61C66F6081089B6F78AE690EE8
:1046A000BEB502A192B6E4B3E2C3C1690AB125ABBB
:1046B00093C2AB6FEB6C98E5967C3ACD2AF2BA6167
:1046C000D220B23D263E5E3A1D942CB88F76D0C2E1
:1046D0003179FD962E4B29375D4E13CA7229125E31
:1046E000D533F6683EDD1A6247CC654FB8A68554CF
:1046F0005409882C894835AFE6E9409752C30A9798
:1047000091DB58C5DA24DFD7B3407C6AAF28E39643
:10471000FAE5663455A0423344A5C44F4126B91882
:10472000C29F95CC75EA0D3FF91CAF1E5943AA8173
:1047300049EC0065A53AAD715CF4CC4CCF15F302A1
:1047400066E6AD65607CCB0008DF95054A40903E8B
:1047500004DC809AD8835CBE9DE15E3A8D87E74C8D
:1047600075D49845881B767E80C5046B0DE4219135
:104770004BD621EE52E40834F7F88C72C159C02BA5
:104780003141061E336C5E8D10EF9B745FC0A1C873
:104790005FDE2E1DB12DABA7091551B180E32BCDE6
:1047A000C1B5F2CE38ECE7507E184B2E43FD2D47B5
:1047B000FBAC1FE7AE03C4E7D034B959E8BC58B826
:1047C00072C75E2AEAF9C014435E6D0CB176B6ADCD
:1047D000D86E2322DD2C56AAC5D9303FC1B02D0A90
:1047E00098C2A1650B0E41B53B8CD6FD94B5DE4D4C
:1047F000F9911282655B03EC6213E9833CD545DADB
:10480000F1BDDA2DE6D242561DEECEAF6E4F9E645C
:104810007ED0FD98BBB2B987780418092775C0B25D
:1048200016487F88F77F4D16E01FB2DA9956EC0CD8
:10483000F0E79CEEAE8113360DF00EF6E7D6B89297
:10484000767AEFA972270884E65FC2BC59CC8C2D1A
:10485000E73882D194AB8585A0613218F17EB9A684
:1048600090FDC29CD0C82357F117BD2F60E10FE027
:10487000DE5F152568B5CA816FE7F11B7E13946C66
:104880000E8F3E799A3DD965781B70EC93BC02F986
:104890002093485A4F237BE9BA47AF30A5F59C5D7A
:1048A0007D393AB775C3F7297E48FDF79DA9850381
:1048B0009279650A8D37356F65BCB88922039129D5
:1048C000013A48138B6D603318A79BD19ABCFB7CCF
:1048D000C2CD2F16237FCDFD62637CC818962712A8
:1048E0001E8A7B53E586F5D724CA44B71AC6ED8DD8
:1048F000D01C1FFD5F1FBA2E7F9C1B5DED604141E8
:1049000015885D200433C8AB2A122EA6473B574CAE
:10491000CE9C2593C23A1D47C804BBA62E4E0AC39F
:10492000BA76686BBB74BE52DC506FED230B00ACE3
:1049300009E2D704EABAF5E881FE1BD5BB309481C1
:104940000C6AEA76329DFACB7954D4ED0114D7146F
:104950005886C9534414A7E5AC75E5E1EC2AD6DBCB
:1049600024C5DFA49DDA49EBDA686FB989A039AFB5
:10497000D2D2377FB2E1EDE0A0EB476E07AC0A82FE
:10498000228FFFA2AB3E1B171C5D6E75FA0E74BC26
:1049900064676C5B75574DA884F4B3580FBEC6941A
:1049A000C2E06628ACB193C2971139BB11507AEAC4
:1049B0006794137301B70AEEDBFE70D8AB8A37D564
:1049C000CDCFE3C3CECA27C507B19E8A084B155D7C
:1049D000F9B159F845A94F42BBB738A5FE1B5F6135
:1049E00067F8751D1A1026C481B7B99868992F7F8A
:1049F0002B6B3E5E32D7AA03F694BF51099C0DBAC9
:104A00009F14769303A4BDBC3657DBD42F6A83B5BD
:104A1000721E7488A9D846C78E6B0551C356A20B67
:104A2000AC8ED0C818E7FA00150B77CAD292388C32
:104A3000EE995B47507DC11015E44DF424D567AF66
:104A400097562D3005A208D6127564B4D4F7D3A2B8
:104A500059E0FDB4543D091A3FAEB2E4493F921803
:104A60005AB9C63201AA401F3979619E74CE9B3D66
:104A70002896086F69570BEBA5AA9CCF8DCF5E4790
:104A8000DC47E894D2DE42DBD06DF07884A4DFC846
:104A90007F22BCC6F1F9F45ED8E406531F9B5D4C3F
:104AA0008CE4F822B3115271074C304364D8EAAA5F
:104AB0003C7661C0548EBD172BCC30B095C8267F94
:104AC00006EAC7853484BE1B1EEB7409441C1E43D2
:104AD000339213E32BD164D42F7CDE70FAABD697DC
:104AE00052E9E76CF7EAEA44CD9CED2AFC3C79E612
:104AF00056F9882B38F419929BA9F4160E8CAA2922
:104B0000B196E84A76958E75428CA6EBC774DEC6E0
:104B10003D9C73393FFB9BC5FBA172D567A67F40C7
:104B20006172F2CF612C4530279B87CE8A3573DBCB
:104B3000F0D42C117F1C6D72C8991936ED4C624F60
:104B4000A05F18644199483F720B844A8A364FC669
:104B500056AA5FB40DA0E102835C73DA6E5E22FB9D
:104B6000537A0588D4D2B5CF5F42A2BD46C7CD8364
:104B7000B937237263988BFDDFE81E8755437EB9F2
:104B8000B0BED60108BBF4093E22CC22FB0EBD9874
:104B900030DE128603C160D8BA643C74FDD5CC8186
:104BA000EE25F3BC3827AEA977023602DB7DAF1BBA
:104BB00031FB9D32C226266E1F7E24888B25230E54
:104BC0005425F2F090CA7A69DEB502D9259C3A4B99
:104BD0008684C4B790A81EF25DA2FE2830B272CFC0
:104BE000F910857A53D677A2F7B3F3AE2F65EEBAF4
:104BF000855B19CC9E9E8548EA508A153F053E7A12
:104C0000B0D988AC78F23B2D147E959C5953512F26
:104C10004FA4A9111FB7330230C57C54D158138952
:104C20007B696792B5462D79751B83DB9B6F96DD9B
:104C3000E83024A584683E333FDC372A8AB87912ED
:104C4000E54EF54536E3673D7D3859AD26103F56B4
:104C50002A6D565EF2383A59AD42512DFDC3A192EC
:104C60008D5C5D28E223BD5B7EA9D0891DA12DB995
:104C7000442BBE1C15AA1E9F47F55AC38798ED41C9
:104C80008252ABFCB104BCFCB123285D2D8FD02730
:104C9000BDA554C2A24D03CDCFFEB943915E029F84
:104CA00099EF713EAE9BED652C9DCC5B6832208BFD
:104CB0001AABCA87D7633D9D70088865B4FED09D46
:104CC000BA2DFA895E44311851CDC5FC812CFD6E98
:104CD0009426F8BA4B4E154D7E2C9BB511149D9E13
:104CE000828FDA3D981D18B4BD2C8601FFDF553840
:104CF0003C2ECC3B3D15B22254A5669BB1651BFBF7
:104D0000FA42F00E92A43FE91F86278EF6859C1486
:104D10001DBA3FBABE73345ABA46FAE48BB4D8AB64
:104D2000BCAE81E2DFC9F2A5E4B0D74EB9C9BC8EF2
:104D3000D7FFA7C85F42C4A8FF1428D2751E3B1B2B
:104D400028FB940D7542258CC122E246B0E58222F3
:104D50009B9B97F98A39F9666522E62A7F1096228D
:104D6000CA8F54E554B3789245DD2A532FF3BF31EF
:104D700052B8197E93BFA98AED23E7316ABBDF7D64
:104D8000C042E43E8C01D318E97417FEC14D158B67
:104D90005F761452C097EC40DA47F65133F654F27E
:104DA00028A671039A0EF5FEE68DF0EABA614B393A
:104DB00033D91BD3B8726E2CDACC581D7AADADAF97
:104DC000D5F871146350573DA396C20A02B2907D84
:104DD0008FB1CB15171EF6CCD9F93FD6F059DF911C
:104DE0003DEABC7AD62E69BE7D67F4B88988892BE6
:104DF00031498F1F69CBC6659927329A0DB17DDF86
:104E0000504F965656D461FEE90956459194B45DCB
:104E1000F0A092F5598E94E1A23A050CA01070CB47
:104E200070D0C48F2A535EB882787837727FB87B8F
:104E3000DD00C8DA2040B658E09C4A816D1B8F75B2
:104E400087C40420A89473417625846B9D196762FA
:104E5000E8504FCE232FCFF5AF931E54B2FFA9BD1C
:104E600049047C21973F3FB2F1C502C625704C052D
:104E70004098D985F1B45A0371DE6971E13FEDDDE7
:104E80008EEB2BAA703E23B730A5945C80A55F08FB
:104E90000B5C7412DE62DE2D0FF449DBAAD13AF20C
:104EA0005ECD10C5540D4F2A8C7C6F8BFD83385C12
:104EB000B0B7346394E2BEB758BB8D5FAC25D6DE85
:104EC0003CC83B41FE5AF0694ED33F362042322E59
:104ED00063270EA944D79553CF9E3AFA549DB3C782
:104EE0004B289B267813FC23FAD16619835EF7FCC6
:104EF0001C5E8682D5CB5F3CB5D9827B46F19FB6DE
:104F0000103CA6723DBDA432716B22F6881932EFB7
:104F10004FD9CABB7D0D40765020E213F3E1E14149
:104F2000A5D4E8E8CDC0C7E73E7426DE2DC32CCC5F
:104F3000A4A575BFAA43FD1C231AB3A24F4E9A2104
:104F4000EE84AD83636606FE6EF50B03F886B1A9A9
:104F5000DD38568B7AE647F2DE018494F3391C740F
:104F60006B4FE81E6B364746005D44E13BDA7BF34E
:104F70002923BF67B410827E990DA3E6DD7FD43C60
:104F8000A22E9D635A972E1D3EE1500CD2AD784162
:104F900083E16D7AC3373B138DD00A04B860B6E065
:104FA0000EBC2EE374BF300C9E4EFE78FA31CF74E7
:104FB0004659F6E3A20530EAF6C02D142D298D4C92
:104FC000BCCCEEEC3CEE27618245581846A6669CA8
:104FD000F216B95BFFE8736C3C2EE1243750DDE834
:104FE0006768D4A84B55382D9561E8D0A204E3A991
:104FF0000A9D66CA1AC53709C76A1808A5F569B5B2
:10500000BD360AA06C18C0DA00439BFEB8A8C4B332
:105010009C5E27F50619BD5BE3E3E85AAD233B1B15
:105020001CBC81554C692F58C421AE9041C552A774
:10503000C41C6AE5A78B5E29D32010F2633C1406DA
:10504000F779F5493C7F273112F469C53002C1D6A2
:10505000C31B5E4D892DCE46C0623621AC2712158A
:10506000A9DEE1DC3A2461E61B7570F20303996B5B
:105070000499F3945E0512667C699DE13CDCC49B57
:105080002FCDDABCE454A88A56403ED808148EF9D5
:10509000A09A85A0BA98C4759E0EA68984F361C1B2
:1050A000D1787054794B7467354E7DC87EF4F12FFA
:1050B000B96F7388940B5A7F60217F86C8DA66F1D6
:1050C0004A1F3EEBB9728345B3551EBC1AE4364EF7
:1050D000D8ED9672292E8184C1ED9797F3297A46EF
:1050E000F58A0CF1E2485CF1374F3B2B46A6AE1A2D
:1050F000DD4D16AB59F7A90A002D88F4AB880614CC
:10510000EBA5F96ED416BD8EFB83DD42E5ED4DAE09
:10511000E378C474D009D1C756B7843C8BE380428E
:10512000F8F6AD17BCA2F8A415284F493C4D7233D0
:1051300011EA1825D1B41F56B094281172F1A42E8B
:105140006F1E46598731100FF357E37ECEB4F6BF7A
:10515000483937B44CFEB5426DAA789FCA95D51030
:1051600074E27074994DDC1F88859FE181AA45F82F
:1051700098095C50CB478896A5A5CF4608EBA4B804
:10518000D663E88E1ECEB97C1FB318F00124B82F69
:10519000D43F333C65DA52F114E9366FD1D4945CD4
:1051A0002F99923AF414D3AA66F4D203E52E0ECBCB
:1051B000B3B4B1447625AE9D305E8689B6B0FBC7E8
:1051C000669E929D3FA73605C564CF8E8869023FD3
:1051D0005C75CCBA818CFAE13F900FE61365193605
:1051E000B238466C0C3F4120A6D69A69A106D01D64
:1051F0008D2563B5DFDD75AD7BEFA008C210D8D17A
:10520000D78B54FADA9083B3B36EF946EF77AD6E6D
:1052100048661F3BA1152CC05931BC5FD0D917A4DB
:105220002EEC29D410294E8F3AB4541EC13B9D3D1B
:10523000E3DFB55F0374FCFA5A18583EA28E936DF3
:10524000F60C75374CD8D979D1195D9CE0B620C0E1
:10525000DA258990B678152906F838CD1778E46AEA
:105260005C06C9CDE4BCBD67ED24B2BBE55BDDFDEA
:105270006B68698BA0730D9BF5A3150777DECBBA1E
:10528000FBAC08AB29D9FAA4A69A8C3290523C1EEA
:105290005C76C834D6F7356EAB750A2A292666DDEA
:1052A0000B5E31976C250652F1EF9F94828187E760
:1052B00036C4CF77C3DF674205E775740448CCA1D5
:1052C000F3E5E8F66567279357A2EBAD65772C52B7
:1052D0009136B69778200F3E9DBC9B2565583217B6
:1052E000793D8974B2FC5248751BA5B3E0F0C9C77B
:1052F0002BD7B727C7A563F8F8AA0862DB77F04C6D
:10530000152053227B0E9F7DC0E23A343CB25049B7
:10531000780929D26E4ACBDA000D105E87670FBB81
:10532000C53D5C02402CB20252C9EAE09853A8FF86
:1053300045E9493F9F8A70DAEF51E159FA92B78CFB
:105340005BB904E118346E79EF640997ABE3F118A7
:1053500035B23A2DFA82E794D68D71E9EBA000219F
:10536000D256F1A38D007D5F558AE52772A508FF0F
:105370005ACC2A690AF97A01047E5D6548A494F33F
:10538000433EB2F89100484B427F2068279B4BD1A7
:105390007612F96A2284026ED6410A5CB4F4D2E72E
:1053A000C28D06ADC6DD32F3A559262EC4A00B4F23
:1053B000261BDFE1457D628155DF113CD927201096
:1053C0000E720C7F073057C4410981D32F84F0F44B
:1053D000EEEEE8D7A0B4CEB07B4368C8C725A19B4A
:1053E0003858C26804A3F8F4E943A0FFB20CFCC328
:1053F000ADAEE6F0B68E1F06ABE350D8AE6D250518
:10540000124F63CCAAFC86A8C30FC01B90A282A82F
:10541000AA1279A1ABAA4D71223249E8554CD1A606
:10542000069CF475CF1DF0DFB7B134031DE58B3F4B
:105430005E5846E3805B8B02BA837D7648107EBA65
:10544000D3BF1645AE1A9316E287EA663DA5CF276D
:10545000FB9DA9CA0DAD7E3D847C1A546B892199B0
:10546000CFC0B8FFD7624686EAF1257FEA7073AFF6
:10547000C15C3689224CDBD9884048451DEF228427
:105480000B3A7CBE03E7B014C3F7932E440D5F9133
:105490008221C2A26E5FA77AFDA7A3A95DB872DEC2
:1054A000A22D1E842AB86DA06BBC4EC682F3740E6A
:1054B000B1C171FE651DCDB7971AEBC44E275935A2
:1054C000A4AAC083E14D9DC902112B64504A32A3A6
:1054D000A9FF49C45606F3EDB62E9F9A321B48AD7C
:1054E000ABC6A1C956F001D20CA3325EEE3FCCCEC2
:1054F0009D2238AE7A9CBCD83A89C402B57CA0C63D
:105500005AA324832B6D7ED5E264D1744DD445D546
:10551000041EC59D9ABB67978F01E9E68317865BDA
:10552000A7E6793EC3667811C0A8D22F34452DA7CF
:105530009157E6C95A960B1BD48DEB9721E1E7DA18
:105540004831713CA203212CC72F2AC45BD04BD217
:105550004DCAA4012358D8FC2302AE909605AB6037
:10556000F7F78090B24061AC4DBA2FE9EF3C14E7F9
:10557000B615F1366A3F981D0591D231ABCD2BF3AC
:10558000F3A51111DE103FFA2B06634F3853C9A75C
:105590008EA2DEFF75C308F311EF14FA61521DBD30
:1055A000CAC1E1E05B7BEF19E10465A09EAF9E5E9E
:1055B00099D5FB56BF775827855E21053AF45FB130
:1055C0001D6FB9AA16DACA41A0A70A2474E61C4CBA
:1055D00039579716CF2C2717A252DCC6E8A436C835
:1055E000D9084608FC6F03E5E4669CB268A210EC9B
:1055F000EBFE949E3AE9F0FADDB06E0CCBA4D0AA93
:10560000232475467936486463D5EC402CDBC755B6
:1056100033892BACB6CEAD4CA9C8AFF7E64D9D4053
:10562000E9DD3F8BB01F19E3B86A30D0F97FEC5346
:10563000408E6E2D76B9DCC5BB32E944A539DB322C
:10564000DC8A55BC915391FF138EF1E58CF14557DF
:10565000559C3452ECE0BB052A6A2EF6A2B7803680
:105660006E73C4A4867D9F7C92F3E66493C6C90BD7
:10567000CF9808D19BF2FAC7B259FC61FB51299728
:105680006EFD22A174BFB9C6911EAFCF86992B962D
:105690006C0297DECE183F0152B209FE3ACFF75E98
:1056A0006C147EB5B69CCD4DBC49E1C189677BFCCD
:1056B00089D9C9853E6A70F70A9999F7529E10B048
:1056C000FEEFA6D622279E254DEBE90673D46C6724
:1056D0000336EC408EB4FBC1B0D768E008DE7A0830
:1056E000759DDDCC811A33203A62A73F30828F2D21
:1056F0002FF82DA544BBF8ACF4D723698CACBFE4DC
:105700000BD4A2DDFB91F04B598D38B96A53A40F2D
:1057100047B280F573201CFBBF430D4E4B87182307
:105720005DC43C14D3E5A739C2CB5E995B711FD031
:105730000C28F2B59547F1F57CE1562B78AAAC35EB
:105740005F960880EF0E9C956183E7F7CBA44F75B9
:10575000AF7193E6F2BC9297CF274F08CAD2D88E8A
:10576000EE093922B2D9DC4B470B2FDC14C28B87F0
:1057700078E135D26F0B423B8FEE888CAC72BADB8E
:10578000FE17688AEB2C3D9138C16B70078DC6827D
:105790008A63D8ECCCB7AF418DC27E79F8436F4CA9
:1057A00077CF5BE98CB956725388179C3B222CC982
:1057B0006F47E090D9BF04DD432516C8284A423719
:1057C00051CA34CC749089C526A8F18AAB6281583D
:1057D0008E8314121780239137292BDF6C1D87824B
:1057E000CC5664654519579FDEC2F3D01CDDDABB89
:1057F00076C9568928E948122501170A0BF654CEB6
:1058000045403E1005766F1D4B5B3F451BE7387EDC
:105810006FAC19ED6CFA73899B338B3A8C0CE322D5
:1058200066B28659F9ED74A2156AF72871F2E2039F
:10583000A83B19E2EDF8B04EA4F07875A0EA53D178
:10584000940CD45A1758EE2F4B8FB774598D0A9772
:10585000918B62658731E512BBF79B261E3A5F8A02
:105860008BF798C806ECBC242A337C0C9D264B4C45
:105870009E5896E945D615935E8B4E4998AC0EA27C
:10588000AB3859A8AE5B76CCAC9C660BD9E401D49E
:1058900045FE938D078CD9E204EECB079153DE07CA
:1058A00045DF4A1A26290D501D5FA341091EAE0A85
:1058B0003F875394D30C3271BA280815E77127CB70
:1058C000D69F975B9669F607CB93D6A17727F61FED
:1058D000D3DFFEA39D4E628F81C4D069A085B984B9
:1058E000C08A2C90045A8DAFD91CACEF0A24F14A1F
:1058F0009FD6E0D633B5EE726B1007ED11156A74C2
:105900005C9F98204B5EAC90CD8AC9B903905FDD57
:105910004AD4C9401A8F649C92812083B7A1EDE1DB
:10592000E4CAB2497F655305CD509B17E45BAE35A1
:1059300037B740AA60A459ACC99AC1B3B3B18307C1
:105940005FF56FE8A01E3B20310390B6B81B5C1CCE
:105950009CB2697D148C883831E4F19C6C454935E2
:105960001B2C90B7F07C7A628669433227EAAC7EC2
:10597000421DA4FCB2A1415DD1ABF62AA80C61AADC
:105980007BFE1AFCBF17D75BF846789E4B1E9266CB
:10599000B5D70658EDA1FF19C152C70C6E4C6FC99F
:1059A0001A53DC74CA1CF45B2260191CA846D98BFC
:1059B000D871130A339F82C15BAF52470DE0984301
:1059C0002E0F3974D1388EF43787EBECEDC99D5B1F
:1059D0007B79125F4FBF1BE5E1343376B45024303E
:1059E000D5B7F8A8371C378F11F8D15FB3D27B2514
:1059F0008D32167A713A82831F35A85BE2786E3C4D
:105A0000F287FC994C8B42D265084FE99C0877607D
:105A1000095B2633B1565A526C216123C34329BA1C
:105A2000A69C2A9ECF6357C00E45EFCDABEBCAA212
:105A30008342D20B9C0ECF942707EC334F8E12D9A2
:105A40008CCB3AF1132C6BD92C949C31E6CEF0FE22
:105A5000E70B4805E337DF242495534BDABDB7B095
:105A600076E66929662593B665106A15A1758307E0
:105A70006E629C24E04E4BDFFFCEA934537C22772C
:105A8000B9E7848E6FB549D63C855952F2ACEA9E8F
:105A9000964F112E2119BB489D233ABFD14A477A10
:105AA00004DAAD75BAC2A2BEA712E837A135D1E5B6
:105AB00040F217626BC7D3F343D6C519B09733E6EC
:105AC000BB25E33923E6605B81309740D328340758
:105AD00057DE29D7E1664647605AF43324184DFA59
:105AE000B04214951159EC629E163CF24C54EE6B88
:105AF000EC1B058BE07B8777FF888AD2F571B85362
:105B00000DE804CAE460AD372BFE6AF2C8E9F04044
:105B1000593505C4FCDD9B28CBB5FC4113BE1112E1
:105B2000F754EC01E4C366947C21FD0B4223458CC1
:105B30000FCB1E41ADF7EAA80BD7E93563A9D38C8B
:105B40000B3602AFB2DFF961C59DD405316864043C
:105B5000A7409BB1EF9C4F56D2BE63845F20B384B5
:105B6000FBDFFE4306E4EA5CB4A54001C5627CA508
:105B7000ABB05164313F02AB25C4A6B4923D470A95
:105B800018AB1F2FA60FD0401B510A896ADB8EA3CA
:105B900010E74198403CF7E1DE00D86D992262C6DB
:105BA000E7C03715706064A4B7A5D887A67C23E842
:105BB000AEBE8821E14D381BF70E17DEA8A3005AB0
:105BC000B7F2617554D201821EBCDCD205FD9E493C
:105BD0004DD58DE60CF35FACBEC6AF1B0B4EEE0889
:105BE0000F84C4B0856C16E50061F200EA8AED7599
:105BF0009996295FB21E5C3570D956639E4E40DA85
:105C0000652ACA14EF012BFA243509B6D900CB8DC9
:105C1000BF5CF594C5FA37EC5D8087831486C3F3C7
:105C200093552B271530EFBAD64BCC7F1C039E5EC5
:105C3000644EA3670C91E2118FEB355175F0EB8543
:105C40004B683A95C553C49B52EB9AC85E847A421E
:105C5000C5B8E595C4602013FEA5F4E714D0848789
:105C60007FAAC4C2B88DB7271811F46B1A6BC07E17
:105C7000B1D80889B3EDDC74CEA321E0511DBBD6A9
:105C800071A630BBDBA99065DA84F2CFD938B45560
:105C9000E042798E3A92084475C9BE080940C7426D
:105CA0007618F60A539EA862FD5EDF6323AD52AEFE
:105CB000154C1D1BA26B7469E555CCF7A3813CA65E
:105CC0003898221E162983C7D5300EC38888D90D6F
:105CD00024101E6929188CAC670E1DCE2765531041
:105CE00068DE133FDE4810F6211E9D8CCAA4913653
:105CF000A45EF8138D47B2EB6C6FB1E5F8B212CC2D
:105D0000C50E430480F6AC01B8A3C3632A333D003B
:105D10001FAF9893AC788F8A909F6D5D88BA886426
:105D2000DFA45B84F5D2362B4468F57354C5C86D87
:105D300090FDA860CFB9B43F1E189DA4949D7A70C1
:105D4000A5F3FEE1BC2B78E1F9E4CFC696FB9CC23B
:105D5000EFCC062E8A02DBEC93803CD80B41B55683
:105D60005E70D27BE1EB506B956E22E69FFBDB48C9
:105D70005A95942F5CE021E58C344601B7D1389FC9
:105D80009FAA0A72A619E3FB264C6688EDCB6A9E91
:105D9000EE5AEC63D06EE06FC6A03DF49D1E2DEE72
:105DA0001B89710653C34A152758B99BE81A19EA8B
:105DB0009063C6E835A23E9BA36DE30135220499AA
:105DC00011BFA895654FAE2D235D559DFDD5D78D8F
:105DD000AAAC9ADEA85B20D721CB56CEBA3B874728
:105DE000FCA8ADEAA2A5EC0E917349E6A280D34AC5
:105DF000DC842388BD12A928533B6F378D0DE21830
:105E0000490F0B478E2D8A8D6B8468606DC9CC3627
:105E10008600225215B7A6066184DEBE8F20CBB85D
:105E2000A3E089F911B73AB99CC8FC6364C8AC2BEC
:105E30004FA1FBF18B67971A6BC9A0280F09E4D417
:105E4000992EF45FFBE0CB666A4A1D1158008F5112
:105E50005D600F8042E18CAFF6224ECF266FBCD939
:105E600023836C3F412B607000CBF9A5929BAE1C45
:105E7000D71DDC6CC0A171F8FB1AB74A5343C46E3E
:105E8000BCF4CE2DA47C19696EE9E28B7008DCD8D5
:105E9000BA77044EC76A03844AFA1180D672295F22
:105EA000D8870903230A3BB644F193B7837EDECD3E
:105EB000331685D09528A59DA7E56E22348EAB4676
:105EC0001498992BDC8D6AD20C432B388FE5B1A541
:105ED000A63A8F21888793A1C95B9C24E625308E42
:105EE00010DF5658084763138CE68F822CEDDEAD29
:105EF0006C899851D1017DED82DE3881091CED5D00
:105F00002C4D223CB111947C8A592DFB698612924A
:105F10007607742B4878E2264CAD9F1DCA7E8B67AE
:105F2000B5F8AB8AB0688B4F59076714F0B2ECF044
:105F3000713192426318BC14E04A3D61B8A11290DD
:105F4000248C1E2E8E2B20B8CC33BDC4DC1CF99BB8
:105F5000E2EDA1714DE7E2A89ED8530BBA3DC9C04E
:105F6000BDE64208644495790ABBB55A5202B07C3A
:105F70002F8F8FAD79C5504AC8309197E20426968D
:105F80003B414129C26033F47A4338036FCC2D4B37
:105F900037A5653FF6578D8660614654666E97CA91
:105FA00074C78A50EA2A140AAB441D849F26ED8EDA
:105FB000767440D32C28BA6234A9D060EFC485B47B
:105FC000912DD93DF8585E7AA698563E0E287BFF53
:105FD000A1C0BDCFACBAEFC27429020907123F833A
:105FE000625B95E6A13ABC3768B8E97C2C5494D63C
:105FF000D0620A59AFE20AABFBC9C614AEAFD43ABD
:10600000909A6CA81B1AF27E9A5899E42F664C6FEE
:106010002D7F5B0E4E3770FD68E7910A96C647E507
:10602000FA98E3F4E7C25DB1DC9805660E02DB3D49
:10603000643A53937356CBA0B9BFB48CDD6F6DE552
:10604000D8B8FFAFE6CF68BD55C0B91E27F9664C7A
:10605000B7912BE0ED99EB5577F0B01F7F6F60F7AC
:1060600078CF2D3AF7E7F2451EC2A6A0C85A1520F0
:10607000D3740C2268A789486EB3166131FB65F7AB
:10608000EF28234730132CAE7CFE91C3A831CFCF2D
:10609000518C37444C89A356595F24BC04B33958FA
:1060A000C65281AAD470A3F4140F2E91B89BFCA001
:1060B0008FDAC494DCD71CFAF3C4051466F788128F
:1060C0002D406B26249BC523418D832796E8A52C64
:1060D000417639D87B6E237B2F00320152195FE263
:1060E00005888B6D4A9C012AA53A98B5E8CF971E82
:1060F000D078C248DA9822818DAB3D0F9AA5680608
:10610000F0EDE9B92F9AA202CDF6B4986277CC3AB5
:10611000A652CC760BFF0C0F478D5CBE608F77C507
:106120002B87AC973DC45744D7C7DA86EFB1922A84
:106130002385182129D7EAB90A9E918D7F135FDE46
:106140003325F1F5B83D3F6F31FB9F6FEF98E41FAA
:106150007B579CD9B60658C814E72396810DC2A96F
:10616000E8CF0105FE7BB5E56B6B0CCF69142535D7
:10617000C8D2B30694A7868D58FA94E0FF494F8899
:106180009D7D19F3A0F8BE9ABE5482E9A6CA0264A6
:1061900082CC149E47F00DA0BD213FFB735D908C17
:1061A0008CC2324516795F3382347077353EEA63AC
:1061B00063F5569D06E49DB11B2E827F1EC8491EC5
:1061C000E1603CE6AC7338D110E2448AA42D1E8B0A
:1061D0000C3688BF04B2CAF7670CEF741688D19CDE
:1061E000743F956B3E1FD21DB2CBFF51E1092EB318
:1061F000AEC164FC6E3C12E74D7F36B20C7537823F
:106200009DCD44A1647EA2BE67169365269013249B
:106210003123AEF41A02F49EADEB0100B7DB13D6C6
:10622000A2378A6E9309C1D8251F3F06B641ED9566
:106230002C33766B18D9E13DE15B2D0F6DD29BD1EC
:106240004728F0EDE938A9CDC866583BE10134474D
:106250004DE6247E89A94244419B08D9DC62D07D69
:106260002D025527D5806F620C9D2138FA52E6EA3F
:10627000B0B855BCD901A087607155C63A0E45F437
:10628000914A3D237BB3526A1295A5F3C8463B570A
:10629000532906AEC69FF43A6D73CBF6373B07958C
:1062A000FD36003EC27FDFF1606EA7F626CFCC0D33
:1062B000F8CAF3468403BB917F8A0D7F86812470E0
:1062C00080C0B2B0EFFCA904C99D30B3E4AB2C058B
:1062D000ACED809AA75E5DF1C51C314D1CBFE2A3F9
:1062E00081534015CF2F00A5A70B33DD4A283DFE73
:1062F000965237721604A384CD8AA161A49A0672BD
:106300005C5144C9E367FD8D53A2B7618DEB530B1C
:10631000C6C8ADABA4E1465A69411110F6CB9BD17A
:10632000EEDDDE5A69B7974CAA54F89800264087EC
:10633000A44C8ACE7E9F7942BEDEE5DF358A6F2C83
:1063400040C576B2AC39FC121145CDED36C4D8C18A
:10635000685C0F0053B0E47B97EAB1BC7B3621AA9E
:10636000CFEFE490B54E959FB534DB5444A1E414CF
:106370007B222A74A4E3D7C22E28DAE41D0A0C94E7
:106380005022BF070672D5DC892DA1BD88BD813F93
:106390003B20778017C290CEDCB3C21EF748201B8B
:1063A0007FE9A21795A40FC2A4F4DCF98E4DA20CCC
:1063B000AB2674F9B9ABD8231494B0FDC0DEA55A4E
:1063C00032795D895631ACBF232F89DF0438612CC7
:1063D000BC93A3023DD1CDC1F1F8D8F238F5074AFC
:1063E000A3454EC90FF14690FCDCBC3B4DE50917B7
:1063F000850F6092FA2087F5F2FA648BD72B84F030
:106400007476E149C1F44C46D855A6814778FB83A0
:10641000ED059A56FCBABE508F9FC2353ABE7F40FA
:106420009FD07CF26BF87598C93CD0FDF291D6876D
:106430005A940A79B05474D0B6E39EB9A8BE5DF1FF
:1064400063035FFAE9885C3CA9BED3E6C4ABB184C0
:10645000DE133000151CD725D00A583214F029E07D
:106460009B4AA2F8BC5C03BB3E17C96027043B955E
:1064700050EF956D60B112B6483BD3C2ACAEAF924F
:10648000005CB10CFEBEF0C7636B8D195C076D7DBF
:106490009DC88B849E9EA963D3042A6E9704480BE3
:1064A000F7009CF403FCE3F746DABA5243F9C4322E
:1064B000AD37BA2A8DCFAA2C77AD251239C0B49149
:1064C000E69DD0F3C8DDB83B86E30A9045CD23B006
:1064D000DD92F8CC0C5B8BCD312F6583C3849B7A26
:1064E000AEF7CE423DE7F831044C4170EFC90146AA
:1064F0000E3AAD30B4C8FA402F1D78467AEDFE72E0
:10650000961DCE8E9C02F6BE7ECA0690A8FFD67758
:10651000C9AA013BCCF5283A5A52FE940B72186C6A
:10652000B4DBBD3D9B1A54BFEA0C755FC7ED7950D3
:106530001F04FFB8FE974790DC1E8B5858BD6D0DA9
:10654000E707502AD93A36AD08A1117CE639EDE7C4
:1065500010FB72D7CD703480DF0B110C264F4E49E3
:10656000BCAA29B7D28ED02175895EA46AB497C718
:106570000896130ACDF91217453D9D8981D08205F1
:10658000F70AC2FCF3ACB6FC0ADB7208BE7C17301B
:10659000E856CA3F6BAAA3B9B4BFBA2B3EA802CB38
:1065A00036F635B43F7487326421F5BC178F499EA7
:1065B0007401464853215D5939E69B66734F651B4C
:1065C000CFCB3520CDBAF7859CEB0F7B69DBDF05A0
:1065D000DD312B2A9A7872F27CB38A696545B569F8
:1065E00095F06C1D390EE9E8C6D3B95C0AAECA0A4B
:1065F0008835C6498E2F52E9D5738516713871FEDC
:106600001F42DBDCA7B6933E92CD4485BF7AB38BA5
:10661000C5ED9994149C854505F4FF93FE4DE16307
:10662000C4CF8DA1FBF3BA51E1BC052C7FAA0DC6E6
:106630002CBFD1ED8A60C5B9AD13119892B04578E1
:106640006BDE3450C90A311F1ECF5BF2B0767F90EB
:106650009C49A49A8094167414869977F8DAE15DBF
:106660002A94462D015D0A7BD6BDCDCEC839F7DE12
:1066700074C91FE3B3333F3F46F16A042926883AC1
:10668000C298308B3F63A7DB14CDFDF27D842DEEE5
:10669000AE11F020B1CE49A38D9D73B142467ED993
:1066A0006EF9FFECA7DB514DDB0A6BDFB383A4026D
:1066B0005500C733217B884B0888EE65C4D0899884
:1066C00054D81A9A0B06215A1CFD16E762A15DC424
:1066D000E1CAA7D3286E2B3F3AEA99774E710F276C
:1066E0001DF72963A13481BC74F13BB2E93FB7B611
:1066F0000F0483547F8773642A268B1D49FB851101
:10670000BE1435D585331389E75BE8CCC9ACD9E92C
:106710003A4FFD18C518508817C7CED449DC788089
:1067200084CB2503905B44387D2C18C8BCE9532BDF
:106730004B979C0913C5F8757EAEF3D84C99BE945F
:1067400003D653CC1AB9DB9BEBC9425147E92C6500
:106750004A7992A8980F0A8CAE26B7DB06F35BC67F
:106760000CC29CB796E3A70DAF83408E2007FF7243
:1067700095F92F8965EE1F4DA862AD33B96077C6D4
:10678000056B0D8274A18AC098DD32710FECACDB11
:106790001F61390E6F613F8D2F53BD01C5BC48830A
:1067A000B1CF1298D2C5CA416D1DED9A50B99676F7
:1067B000E3629F1E7A2862599A48D1ECF1BEC1A5C6
:1067C00060EDABFA183FDDF9FF2512B4A15B656CF3
:1067D000805D55F273ACA11F7503269C9AB07A8731
:1067E000FFB02D6994F3D25E2A5886B7E9BB87368D
:1067F000F056B33F85EE939427D54AC1C63361A0C6
:10680000234A10FA55ED41DCF534D18057A710F535
:106810006B36F5A84EC89FA8292FB592F2C9E1049E
:10682000EC393A7CF2C8C4A9BD1D156855022FB9D0
:106830003CE869EF609F409DAEB04498996CBD4FB5
:10684000FE87AA0FF7FB82704C8884CA9B9B381383
:10685000AA066C1F3096110751E217F10D71115104
:106860005D617142AFFBBFECCFD40C0AE3FAF525B2
:10687000993ABA5F79284B61FCEB1811094D5261C6
:10688000F3B7FBDB86BF55DE8C8509F4962ABB2D5A
:10689000CB9074739DA2B1FD28E643E5EC1E6658CB
:1068A000837E72AE932DFABECF44B2F9CD37AB2DB5
:1068B000D0D37BA107EB859210E9C8022406F8A487
:1068C0003D080D930FBF1E925C83DBFBDE0F8EF342
:1068D000F12EE6529A5912D9253F0DA0D8FF4ED677
:1068E00044D62DC9D461CC3E7179299609EABFAD51
:1068F000AAF3B9943E6E5DA7480C62320D24CA4FCC
:10690000D7B07027349AD041E115C429207C63EBBD
:10691000BAA759D456006410AC84538D00DB5F9F36
:10692000151448FAFE56720E9A29BE87CB5920F5E7
:10693000DB724B36152BCC2B8753AE832418981B58
:10694000052955DF20653D71DFA9566A2F739F7AAF
:10695000A7CE4780DF6D00CBCDE41A13B6A7F22097
:10696000D49FFE3A0C338501B26F3FF37BD2B8BFA0
:10697000FD3E0A902D4A56E80E36A373FB77B9DA2E
:1069800050E6B198E7CDEDDA2EA6E9FC6B896B5C99
:10699000D6BE53D8223BC637A56D111B7E5F8D83B3
:1069A000CF220B11CDD1CAF5ABCB1B94FDE1323216
:1069B000401CBC65DD476E4341F89748D4D199C56A
:1069C000D4514034277C2CBE046EAA44FFD103D995
:1069D000CCDF34094F74CBDFB4BA31FF849BA4E51C
:1069E000364175AA4BF2C02E960C81A4B8AC79FA48
:1069F0007A4A5FECB668039C30E41D9CFFC5C794DF
:106A000047F68B6BDDA6199BDF829A64F249F6B1DB
:106A10006E627A39A0A1299B35E5FC6607BCAB5BA9
:106A200028AA8D7A4EB8609459F539C105DF22A99C
:106A30005DE16299AF58AB65FD3BE4CBDFCE370B30
:106A400085DDF116AC199D5D24AED79166A343F99F
:106A5000CFEF01EFA6CAD73EB6D02990CA4939E494
:106A60008660083DA955415CD7B268E72077EAF512
:106A7000EC0B505D905C0FC5B6ECB67842F0DE19B9
:106A800092C1AD5DF9D95B486DC0DC0CA85716B951
:106A9000DA221D121807BE4141D2CA94DA3EDDE166
:106AA0002DADDA3CA447D9E781F7DFA1DA3C23E436
:106AB0009037E24BE4D5808001FBE44B358D60F9E3
:106AC0008E99BF97211F552A97A98D60DBED187A03
:106AD00009263ECA789FBB9837BAB34E87BDF908DE
:106AE0001D88DB7F7C9DB3CBFE50885BFC7093A23E
:106AF000260346600B4DE209363A1FD8C3EAAD2E95
:106B0000C1DFD3CAE6BE83D9E03F034A1FFDE31CC1
:106B1000F046F65499FBCC1594BEC59D232649D268
:106B2000C0CA5CC0AB09CE3AEF4A62938FB4447FCF
:106B30003D6342BEE5986E2D7B3AFE18AFC3E74237
:106B40009284AE1C049F6465B579BFCBEB3D2D0DDF
:106B5000D0CD85BF44762156CCDCD4AA50D91912A9
:106B600035C1F252BBFBADE092614E61934D709422
:106B70006BC9F086ED38AAE877F93F26198EEB66E7
:106B800020DC2BC1CB4738185B4EBD86AA1A66F0B5
:106B9000F2BFFCFD76887B5F26CB4F5106C8F7CA53
:106BA000243873F0DEEFE10BEEBAC0A3AB0BA9F112
:106BB000B7BED0B9CFF8D8661C8CD34E3876C3BFD9
:106BC00079251E7C5C8CAE71597810AF9AC9F4F5AA
:106BD000939D7D902C5AB05679628BF9A8C0695D5F
:106BE000B4C78EDB6EB39F6E41643319D3A863E6DE
:106BF000CDB50E3E3D448E6FE1521EA4B79EBBDC68
:106C0000281E100140842298600D2A96089BD78A7E
:106C1000171CC88CFBAB0E89AAFEF24EE042AB58A3
:106C2000755347783E29A3C5DE82157E143DC6AE56
:106C3000EB6B548CB3E0B7CEFF1EDB2DF6B0A36731
:106C400089EE57B33AD2445552AF12F81BC26C4B7F
:106C5000ADF14E7B0E111F79976E358975AF0B2103
:106C60006A638D02E4ED8098258527512DDB22E1B2
:106C70009985E58F84417646D11E785CA67E79DBC6
:106C8000A6659C28D8440A4C3A400D5E237ADDF074
:106C90000957ECBEF756A99AAEE1663F5F76C2741B
:106CA0007C2A56FC08C5FAC74B74A33D70A25AFD56
:106CB00020E3A33E3DAE09DC14E6960C7AECB498D2
:106CC000B3919A81EFFDE486185D1B24B5ABD3B276
:106CD000B42879A53C8173DB6149D413E3309B1C54
:106CE0003E7B07FD90E4439FFF898CDEC296FFDF69
:106CF000C2085B24BB0F2F1B5F5B74D9CCA21D2283
:106D0000EC0850382A47E1BA57487FDA2966A7408D
:106D1000337FB8F2AE87147AB691DC0DD89413564F
:106D200099E865DC7E26D70B10D2306827DEE5D9DE
:106D30006CC520EEF381FBC0674428508DB803BFBB
:106D4000FBB81A2D9111727CA299D2A274EE02F4B2
:106D5000E16D39D9FC5A4AA67E609034F6319D55D2
:106D60008E41CB5F97A670AA2AC02D7EB738D97EF8
:106D7000057923A41A999F1A0B9C75112D0CF5C83F
:106D8000947B4ACF687FE7AD5E7BD812874786CB7E
:106D9000FB1664589BA4D7E2BC671B7033837B6FE0
:106DA000704CABF52A8C6DCB8061B49062E72E34C9
:106DB000E8CA9471F91EF93F8C32BE4FC3B4A129C1
:106DC0004A173938121F3B915996117BABF9BA6BB0
:106DD000EFFB2FE492F30FD4756C4FA899E9AD093E
:106DE0008B1B1B936FC1A3A93EB83BAC9B3C6C872C
:106DF000556E50EABED8BA256BB93412BF944E878F
:106E0000F24585C93177D08F638989CB3FCF7C2FFD
:106E10001077631EBFF226EDD56D7A9E708176D90C
:106E2000B572454F38D06D2CECAF57FCBCCE7F7798
:106E3000932EB79743ABB0F6E76CD0BEAFCA0070E5
:106E40002A20C0C6A9A0F6F6E9F88E40DA590F4A02
:106E5000F5AC66EC46B267F66D30CF5134B4DC1158
:106E60004DD3E45C588D91E015C29B951AA08F918B
:106E700009A34F27CBA78244C2B34E87F6F5246DF2
:106E80008327FF7EBF004D487675120A21F46C956A
:106E9000010352F6CE50D58F4ECEE3FBF207B4B2CB
:106EA000767E0BC85B4A8F54D2894F807728E1DD0C
:106EB00033BDE177864073BC56EFF6DD7DEBAC3C2D
:106EC000A8143766610C413BB91A2FBB1F57967740
:106ED000B33839963525304C02DF0CEAD7B35E87DC
:106EE000DAB388C759739CFAEEDB72637002BDD6C1
:106EF000DDE92B25347D37A9C6E0FF53930C74766A
:106F0000942BFC187E228073747E84021720BDC6E9
:106F1000233B0A01ECA988CBFBD86336E702DB45AB
:106F200056F8E346A8929ED828BE32226A072DBAA8
:106F3000966260585448BCC14669142874CEDC7906
:106F40004C41E9D8CB82FE67E774F1BAE9DD274E00
:106F500096BAE52F15AE131B0C12984D1F28E17839
:106F6000EDD4F07554C7F6E4B62A9E073EFD01A99C
:106F70003D5B495739CA459B981B316F158F7ED0B1
:106F8000AF77B2A87999D423F892B4DBB5DBF7AE2A
:106F90009F3001A712013466595EA6964547E6C4A4
:106FA000720027605107C12B170DC72CB76FDFFD8B
:106FB000D05E29407ADAEA99D5702F1CD1463397F2
:106FC000D40749E3CDC3E7B27056C5D053ED274986
:106FD0007F3EE40F49ACCD1B7155D7082D9F5DEC6A
:106FE000206E60B94252DFD638F80B68C19B43A1CE
:106FF00089D504914AF7CF19BC4D6595CA8575EAC4
:107000002C7BB9D272769791DC6BB8B2B1DD20E2FD
:107010009EB980939652C4D3EF02A69AE6C7AAD22D
:107020005D4219098E6AC1E5BC0A41C0D0EE39C380
:1070300074BDF1181B6AE1518F21B826793B113DCF
:10704000C31DB5D391B5EFEA28CF50F2B245500039
:107050004B33707F7ADFD7F5C5AF12BB0A9D3D0772
:10706000F00AB5373F66191C784872152917D8AB56
:10707000E0A291F0AD6B8BA1976E9D8D3EB42A1569
:10708000E76182C4475287D44E5B780EABC093C68B
:10709000CD97EEC8946AA6D41D04F72EEB49712251
:1070A0003609F7601942DF9B77F6C8A69B4C5467F8
:1070B00007A0F4DF3DAC736D0C538DC6AD4EC770A9
:1070C000C990A0EEAC6C02F15D08234F9803DB1B66
:1070D000D5F406630E4F2647788F8B5A39B6FF7664
:1070E0007F0391A272BC76055A5C0DD55937E24DEB
:1070F0000B52DF26574CB75A2BF2925B8117080CC4
:107100006631408B5FB880DBFC8A2C87A929B030C0
:107110004C3747B12AB4D1E965C87610DA6407AEB6
:10712000C45E5C5130A538EF2B53E43E2843936690
:10713000E78490FEE94A6A8452BA1AC382A24E08D2
:1071400007E40BBA25709A0F7A1AE5BC64303F98B1
:10715000AFA3F6C1305959658E05C85310E743B740
:1071600009B10F081D84949E6425EF60F4E6CDFA02
:107170001DFB541A7FB0BEE35F033493EB3B396AC7
:10718000914CFCA139371B7BB1C120B3AEA19B3818
:10719000597D586041EB2247504A49407694247902
:1071A000A3BF98FCE81F385AEE2A6159007720AE39
:1071B00016D77C6D88291D280B66D4FD9E70424F22
:1071C000986042D66F4AA503DCC47E8C0DFA13EC9E
:1071D000F3397D13F0C700FAC3C730F9B0C699443C
:1071E000DF3209421B1B3D878BB7E292A0A5710FCE
:1071F00064D03861681FEA23638C3D0C46294AF746
:1072000011E22B446EC4CF0E179C48F45BEBD9A35C
:107210009EC6B41FE92D265F2BA45AAF01E70DCE01
:10722000797AE2FA679A249A9A909E829252AF8370
:10723000B2CE4B5B53F2A4B2F48D2EB104D37AA13B
:107240005964054645D2DF90184D49FA834E999C02
:10725000A81C532B6F0ABE499DC7FC75522C8DD8B4
:1072600038A209803E12861049A52C5630613DA4F3
:10727000080328821DA2B7241732C5BB28AF76FFAA
:1072800024037740597ED4C67118A17F0A7F7BB151
:10729000C0B185C5C599647209FF65414B5A8C64BC
:1072A0000E8E0A6C55521B70924B97E34CC5979CFF
:1072B0003516835F47710926408754B0F94B7047F4
:1072C000313378858DBA14368BF0E4145BAF8B4282
:1072D000341509395DFCD663721F5173BBEAD36262
:1072E00087F75BBB934426BDF45B516DA046F25F0C
:1072F0000B05EFC6D13C52EB89919DB8EAA584629B
:107300002CC3552453BC8E52E27047E677E0E08FE1
:107310004BB63A359011CE326A81BC2EE454C0C9C6
:10732000360AEF50213CCF3111BC6184511D75EEFE
:10733000DB079BD4A9E146B951A62357DB96F71288
:1073400032DBA4D4AC7A5B2C9D5EF28220FC067307
:10735000A81ED70468D75D7D05C78D282A1ABF23CC
:10736000F12AF6D80954CAA91A6F0F3AB4495886B7
:10737000886333524E47AE996A9C7510C44FE91C1E
:10738000F64081660059D9E6317B505EC666492DCC
:10739000DBF8CF35FAED6DC54331D5503C3103BC38
:1073A0002A50EF75973CE88700C4F9DEBEEDDD7723
:1073B00071290B4D6A57DEDEE07E1D9F8AD7D9EF1B
:1073C0001FAEBF5605348FCA35486984383070E81F
:1073D000FEB5F14B309DFCD07BA3B16BD7094D9529
:1073E0009BF0A28185DC0FBD4853BEE24555E01CF1
:1073F0002C8ADE6977E7EB51C6089C54861C541D25
:10740000C0189B89BB02388C56A87CA49F98148B0B
:10741000133945A956781D0E60B447DFF7457351FF
:107420001E2B6CF863D7925205F9611B1511A2D37C
:1074300060557C2EE8EC8FE9E4D665D3C7A8D0155B
:10744000BE9B7C5E682C64CACF20977B3F2939E3C2
:10745000474221BBBE147D10958BA1CB725543636F
:10746000EC11AC51A5A9838FE413F46FEA41E870E5
:1074700082A23C6459AE97706171A759053D746E44
:1074800073D54D89CF6E3FAD39B2C956CC9B3F5EA7
:10749000CAF1D4F4ABDD262C2EE7561CD7557F70ED
:1074A00062A295B29794565B19381700678B2A9C95
:1074B0007AC2685DA6585813D2ADADED3548574134
:1074C0000C466B120B7313441B776B312592032F01
:1074D00087F01BEF3E2B465BCEA6FE55D71884D314
:1074E0009B8C2B559C5041D02CDA8D2B21113A4E80
:1074F000B426E64AB96883CBDBE753D91AA9D27E12
:10750000C182A33902C38012D00C22DB3C93E61B5C
:107510004A9E48E109EA16B68B3D10D932A28A4A42
:1075200005FAF45D153FE49A15357FD69DF2C0E566
:1075300060E1130843EFB565C92F74713BA3AB201D
:107540004A78A4DAD1DD58EFFD61C5A0DCB40A5257
:10755000B5FCF512CB4D98C2E5AF947BFEE94A9994
:10756000BBD15347A9C1E3374B6CEA0BF5AAD01E38
:10757000FCC6FA8EE3EE4D26EB4E28FBDA9AAF6A94
:107580002193F64E5F182F7004C508930942519657
:1075900008550C31130F1BE4450243E2FC0A0E06AA
:1075A0003850502080ABB712D46C70B53D4BD772B9
:1075B000B37121C5D169253D38C11C7E162838D943
:1075C0009B43DEF37F3A1C142A1DCA592D09909360
:1075D000C92135DC6A2C00D6BAD4B115EC531A781F
:1075E0004473AAE4354289A21136827A322B86ADE1
:1075F000DCB2052E2D73C916EBD4FC3ECDEC223A3D
:107600008281FECD2CC30A2CB9D69D7EEB82FE482A
:10761000AED67D9167129E5A2ED7A1AB4C8D1657D0
:10762000B3461523973F6AF69EE5093B822B147EED
:107630001A413D6A4EA09151D3609C1A078950CBE4
:10764000DAB225A2CEC30FF9CCDC47F7B441A6A924
:1076500082545A59B63311FA17FE57045D145F9CD1
:10766000EE36C9E0D81679372167F08CF99A2F5B8E
:10767000E77B0234DD8B3CE651771867F7A9BA0542
:107680009461C66B219FBC7A0D8A2F6708240A3447
:107690004B5255FB377C8849D3FD9603E24408D909
:1076A000ADF07B83BE46D82D13CF6A906F6E799B69
:1076B000DAF3727587561391DCA30B6C3A315318C9
:1076C00008C9867DF259311B7A2F22A7DA9AF5E193
:1076D000FB7EA994A55D9225EB3DCA82F4C502AB61
:1076E000D56479DFA3E2BD3F52B15A09D72BDFEB56
:1076F0008E48B2E12167C518BD348612771E219EDF
:1077000033D2158CB97FF9303D33E55B05FFE35388
:10771000F4DF78CDCA2CA9AFEC551A6AD39AAAAE79
:10772000DE697B58A7369EAFC7D0B0BEFC9A4FBD6E
:107730005FAF095198AF394FA29FCCDCA177690A9E
:107740007599B834CB74989D6C2A9E665F7D6410E1
:10775000DD277F39004FF342A307E43762616CE90C
:1077600022D9E886BB45F8A87FDA0218FE473F2AEF
:10777000AE4CFF87A8703454A9BE58BAF81AB302A9
:10778000D839B00E84B5C6132CB7EE70252B838A7A
:107790003838CF03F1984B746667363E7F52913686
:1077A000D0E6CCF6E6023400AE09A9EFB7D94A9B81
:1077B0008232D287E1D0BB58C1A2B1B50754675716
:1077C0004D8BA7A30D76273FC028EC8228DA1D9C9D
:1077D000ED3B27BA041FA6E892F3DFDD75AC77A670
:1077E000CA36B19B3E9BA17BE6FEE5080213BF9D16
:1077F000FC0E0B975DF5020720A389CEA7B1394493
:10780000ACD9ADFE235AE6124A7BE5590B4E0298DD
:10781000B45F31D1F4A135732D9B254994C10CD1AE
:10782000453FB19ECBA27B6C793CA9F97B33E2B892
:107830007859DDB78DEE99704F1EACE4F27C3CCEEA
:107840003AC798A97CF9E122C24DE43A541AD8A06B
:10785000977553C6C67B858C49E6E37F27D61BF513
:1078600076FA89AC4E9824BAD63220F1434F4E5F57
:107870007F1BA03AEE86A4A50E251AB262632DC521
:10788000387DA7DF5E431FD8BA8A21664317C0F050
:107890001C50F7A1304101CA0E83116E22E596DC1F
:1078A0008173085312B330E9D45562B89F97C975F4
:1078B00018F3F029E891765A229D83F7FCB82253F9
:1078C0007AB4525EF7E6051D0356EF788EA01537A1
:1078D000E17AA30DEB10CA1603C1F5CA8476212CF8
:1078E000EA39318811BAA966BDFC67D49EAF928887
:1078F000F67496C346C948923616F22D74F3172FC4
:10790000F7E8230CE5B9CEE16E5B061C3151FCA60D
:107910004D677D59F9877152B38DA0F918B3029262
:107920006AB1643D16482DD90DCCC9A13F3165A37C
:10793000251F7EA37EF8FB92C3257D3FC26BA6FC6C
:1079400089B3351F221C731BF8E55ECD55A8E452A0
:107950002F7383B66BB47F008E44E77D3A58FE1ACE
:10796000DBA1DB382D8D86A14EAF0D751357E3A932
:10797000CB5BE8BD7D3E829AD57D17C922A6ECB1CE
:107980002C805B9891C1281DDA2401E1080AE38B61
:10799000B1C0C8B2B3A6B41BB95D98B25E2128329B
:1079A0000486A29FA5DFCAAA40750457493AF64843
:1079B000146DC01BA786FCC31E0039426DFA0AD99C
:1079C000BBD504D157FA8F7CBDF7BE4CBB099CE1F7
:1079D000AB58945C3D15A9AFA9A8274549671E0877
:1079E0004CC49C16F3618452562BE467D31E44B7F3
:1079F00091FD098652FF274017EED5872638F1D82A
:107A0000A9DABAA796E6C07FF5460B89EA28A994B9
:107A1000F5B55C84274EFF904E9FB57D9C59A6A07E
:107A20003F979D9BBFD6D26B2A9C4CF9E1CEE3C514
:107A30006B04049532CD66203CBFAF826D46A6270D
:107A4000F50B3C46E34BC63E930AFFE840F19A9B98
:107A50004F74968053C38EC4F0BE8B2BB82C60221B
:107A6000FE5852724B5C27A850ADCC475CB72940FA
:107A7000070DFD44E3810C0AE22D57CAC372D3C03F
:107A8000F945ECA4F9E494E8B5B251E2D2FD003D29
:107A900024FB5BF4197B5F89C449D32100722D97C5
:107AA00020A31D442159893E8741AA5D265B8A5047
:107AB0007F1FF6291C3C7888AF435ADD1A1933E43E
:107AC000495797481C416E67DD988EC0436AC3A032
:107AD0008C67F2932770E4C29CB18BD6D143FBEF45
:107AE000A8ECE70BBAF385C8914A116B5867A72930
:107AF0003C9F13693D359BAB3F2C4D8D9873FE32F7
:107B00008F5461A9E6E5BE7E3EFCA7158204A28DD6
:107B100096167F123418EBCE4DB59681469BE772D0
:107B2000583371146D8A5E508FB7AEDF926620FCB9
:107B3000FCD80B98E3D818683D7C4B3A9A2FCF4C71
:107B4000D49340C6077D1939A4995729C36D67FAA4
:107B500067C841F350B79DB0D1E2F6C95A694F7179
:107B60003737CB83D443D5729B493B4D63ED9EA4FD
:107B700050FF99B66023DBC1ABBB2ED0ABDAB6CDDC
:107B80006DB534DF5BBBCD401F28A893C44D32A137
:107B9000225D044E9DF392D88777A39730644BC043
:107BA00038E9B8EC587C79937078E940FFE8B299ED
:107BB0008C77B33E5567536AD000BFE4E7BF93B0FC
:107BC00093BD36C12886D1F523E73B973F1A81ED57
:107BD0009AE12899DC7684D3BB1D468FE3013D16DC
:107BE0009DACFF23E584E960EE263624A190D3CD39
:107BF0001FBA9DBDFDE5D19D812F77D5722548D453
:107C0000850A7B171B20549BA3E79BA703BA6D0B28
:107C10004B67C69062E8A610FA617CA36DB9B17992
:107C20005AA4FD7D0FBF642B0C0EF3E31A67379542
:107C30000E597728E9F11BA164EDBB4067852B2B1A
:107C4000EDD9DA8DCA0AD36468F7C7F4C09CA96677
:107C5000D215A22948E575EDDA2462FE461C44845B
:107C6000901C870B8CF0F185CBADFDCE12C99EB672
:107C700092D826A9BFA45CF451B50BA5854127DC99
:107C8000346C45BDBA0FEDBA50D44ED10AEF6F6CCB
:107C90008D57FB514BA0DF4FDA3FB7F92D7B89178A
:107CA000D065F826FE4CEDBF1B5070371CFD5A55B1
:107CB000C4DE8DD7FA801CE65B68031792C88FCEAE
:107CC000D6067A742048DFF23D28CACC3DE1642B09
:107CD0009F133D0468FD0155DE97296D97C3A89950
:107CE000A10EBC1075EC8627D7B15FB84E28A3D182
:107CF0009494110C40CA24BAD633AF4C3E6913A4F5
:107D0000AB7606FDDC6548D19819FC559E4ACBB28E
:107D10003BEBACFAF0C80CFE5517EC5F8E7248DEF8
:107D2000987AA860269C93A10D3C12AB39B5E31C50
:107D30005A2D25D6BB53AC3EC1BAEADB31BC543E0A
:107D40007D539938AD8E411C08E4961C96D7249833
:107D50007B5F616942AD1C0418D024E140897C2816
:107D6000C69EEB369DE679B3B34BD68A7F59BEF7F4
:107D70004BB6DD43D3E779CCC12C78A717291E5C1D
:107D8000ADD9DD091541EFBC8E99E80BE9198215D3
:107D9000398E577AAA5F33FD0304050A08060BFFE4
:107DA0000209070D010C00FF202569202569202507
:107DB000692D256900202025633A256900202020AF
:107DC000205F5F7C002C0044697370206F66660D35
:107DD0000A00555345520046004700424547494E68
:107DE0000052414400442E4D590043005052474D2B
:107DF0000055534552202020006620200067202097
:107E000000424547494E2020202020005241442076
:107E1000202000442E4D5920202000432020200007
:107E200005000000FFFFFFFF4D000000E9400000DB
:107E3000000000006D10000001410000064100003C
:107E400004410000FF000000310800001041000064
:107E50001A410000B8400000000000005106000078
:107E60002C410000064100003841000000000000E5
:107E7000F10600003A4100000641000046410000C2
:107E80000000000089080000484100000641000091
:107E90006941000000000000190600006B4100006D
:107EA000064100000F000000F4010000040103017E
:107EB0000201010411040F04170416011801000047
:107EC000F17D0000F97D0000FD7D0000017E0000D5
:107ED000D97D00000C7E0000137E00001B7E000098
:107EE000EC7D000000171B243E4253697505020516
:107EF0000804080B08040405010504090809040620
:107F0000080702060204020601060407010308032B
:107F1000040C080D020C0203020C010C040D010DEF
:107F2000080D0408020808070802020704080108EF
:107F300004090209010A080B020A0201080A010ADF
:107F4000040B0102080204100811021002110810AB
:107F50000110041101120212011302130812080F7A
:107F60000812041301130414021401150215081455
:107F70000817081404150115041702170119081A27
:107F80000219021602190119041A01160816041B17
:107F9000021B081A0818021A041B011B04180818EF
:107FA000040B04202020202020202020200000007E
:107FB00001000000D27D0000D77D0000D97D0000C7
:107FC000DB7D0000D97D0000E17D0000E57D000043
:087FD000EA7D0000EC7D0000D9
:00000001FF
